Archive member included because of file (symbol)

C:/Program Files/Microchip/mplabc32/v1.12/bin/../lib/gcc/pic32mx/3.4.4/../../../../pic32mx/lib\libc.a(memset.o)
                              output_pic32_ssd1963\FSIO.o (memset)
C:/Program Files/Microchip/mplabc32/v1.12/bin/../lib/gcc/pic32mx/3.4.4/../../../../pic32mx/lib\libc.a(strcpy.o)
                              output_pic32_ssd1963\FSIO.o (strcpy)
C:/Program Files/Microchip/mplabc32/v1.12/bin/../lib/gcc/pic32mx/3.4.4/../../../../pic32mx/lib\libc.a(strlen.o)
                              output_pic32_ssd1963\FSIO.o (strlen)
C:/Program Files/Microchip/mplabc32/v1.12/bin/../lib/gcc/pic32mx/3.4.4/../../../../pic32mx/lib\libc.a(general-exception.o)
                              C:/Program Files/Microchip/mplabc32/v1.12/bin/../lib/gcc/pic32mx/3.4.4/../../../../pic32mx/lib/crt0.o (_general_exception_context)
C:/Program Files/Microchip/mplabc32/v1.12/bin/../lib/gcc/pic32mx/3.4.4/../../../../pic32mx/lib\libc.a(ctypef.o)
                              output_pic32_ssd1963\FSIO.o (tolower)
C:/Program Files/Microchip/mplabc32/v1.12/bin/../lib/gcc/pic32mx/3.4.4/../../../../pic32mx/lib\libc.a(puts.o)
                              output_pic32_ssd1963\Application.o (puts)
C:/Program Files/Microchip/mplabc32/v1.12/bin/../lib/gcc/pic32mx/3.4.4/../../../../pic32mx/lib\libc.a(strchr.o)
                              output_pic32_ssd1963\FSIO.o (strchr)
C:/Program Files/Microchip/mplabc32/v1.12/bin/../lib/gcc/pic32mx/3.4.4/../../../../pic32mx/lib\libc.a(strncpy.o)
                              output_pic32_ssd1963\FSIO.o (strncpy)
C:/Program Files/Microchip/mplabc32/v1.12/bin/../lib/gcc/pic32mx/3.4.4/../../../../pic32mx/lib\libc.a(printf_cdnopuxX.eo)
                              output_pic32_ssd1963\Application.o (_printf_cdnopuxX)
C:/Program Files/Microchip/mplabc32/v1.12/bin/../lib/gcc/pic32mx/3.4.4/../../../../pic32mx/lib\libc.a(sprintf_s.eo)
                              output_pic32_ssd1963\Application.o (_sprintf_s)
C:/Program Files/Microchip/mplabc32/v1.12/bin/../lib/gcc/pic32mx/3.4.4/../../../../pic32mx/lib\libc.a(default-general-exception-handler.o)
                              C:/Program Files/Microchip/mplabc32/v1.12/bin/../lib/gcc/pic32mx/3.4.4/../../../../pic32mx/lib\libc.a(general-exception.o) (_general_exception_handler)
C:/Program Files/Microchip/mplabc32/v1.12/bin/../lib/gcc/pic32mx/3.4.4/../../../../pic32mx/lib\libc.a(default-bootstrap-exception-handler.o)
                              C:/Program Files/Microchip/mplabc32/v1.12/bin/../lib/gcc/pic32mx/3.4.4/../../../../pic32mx/lib/crt0.o (_bootstrap_exception_handler)
C:/Program Files/Microchip/mplabc32/v1.12/bin/../lib/gcc/pic32mx/3.4.4/../../../../pic32mx/lib\libc.a(default-on-reset.o)
                              C:/Program Files/Microchip/mplabc32/v1.12/bin/../lib/gcc/pic32mx/3.4.4/../../../../pic32mx/lib/crt0.o (_on_reset)
C:/Program Files/Microchip/mplabc32/v1.12/bin/../lib/gcc/pic32mx/3.4.4/../../../../pic32mx/lib\libc.a(default-on-bootstrap.o)
                              C:/Program Files/Microchip/mplabc32/v1.12/bin/../lib/gcc/pic32mx/3.4.4/../../../../pic32mx/lib/crt0.o (_on_bootstrap)
C:/Program Files/Microchip/mplabc32/v1.12/bin/../lib/gcc/pic32mx/3.4.4/../../../../pic32mx/lib\libc.a(default-nmi-handler.o)
                              C:/Program Files/Microchip/mplabc32/v1.12/bin/../lib/gcc/pic32mx/3.4.4/../../../../pic32mx/lib/crt0.o (_nmi_handler)
C:/Program Files/Microchip/mplabc32/v1.12/bin/../lib/gcc/pic32mx/3.4.4/../../../../pic32mx/lib\libc.a(_iob.o)
                              C:/Program Files/Microchip/mplabc32/v1.12/bin/../lib/gcc/pic32mx/3.4.4/../../../../pic32mx/lib\libc.a(puts.o) (_iob)
C:/Program Files/Microchip/mplabc32/v1.12/bin/../lib/gcc/pic32mx/3.4.4/../../../../pic32mx/lib\libc.a(_fputc_simple.o)
                              C:/Program Files/Microchip/mplabc32/v1.12/bin/../lib/gcc/pic32mx/3.4.4/../../../../pic32mx/lib\libc.a(puts.o) (fputc)
C:/Program Files/Microchip/mplabc32/v1.12/bin/../lib/gcc/pic32mx/3.4.4/../../../../pic32mx/lib\libc.a(ctype.o)
                              C:/Program Files/Microchip/mplabc32/v1.12/bin/../lib/gcc/pic32mx/3.4.4/../../../../pic32mx/lib\libc.a(ctypef.o) (_ctype)
C:/Program Files/Microchip/mplabc32/v1.12/bin/../lib/gcc/pic32mx/3.4.4/../../../../pic32mx/lib\libc.a(doprnt_cdnopuxX.eo)
                              C:/Program Files/Microchip/mplabc32/v1.12/bin/../lib/gcc/pic32mx/3.4.4/../../../../pic32mx/lib\libc.a(printf_cdnopuxX.eo) (_vfprintf_cdnopuxX)
C:/Program Files/Microchip/mplabc32/v1.12/bin/../lib/gcc/pic32mx/3.4.4/../../../../pic32mx/lib\libc.a(doprnt_s.eo)
                              C:/Program Files/Microchip/mplabc32/v1.12/bin/../lib/gcc/pic32mx/3.4.4/../../../../pic32mx/lib\libc.a(sprintf_s.eo) (_vfprintf_s)
C:/Program Files/Microchip/mplabc32/v1.12/bin/../lib/gcc/pic32mx/3.4.4/../../../../pic32mx/lib\libc.a(write.o)
                              C:/Program Files/Microchip/mplabc32/v1.12/bin/../lib/gcc/pic32mx/3.4.4/../../../../pic32mx/lib\libc.a(_fputc_simple.o) (write)
C:/Program Files/Microchip/mplabc32/v1.12/bin/../lib/gcc/pic32mx/3.4.4/../../../../pic32mx/lib\libc.a(_flsbuf_simple.o)
                              C:/Program Files/Microchip/mplabc32/v1.12/bin/../lib/gcc/pic32mx/3.4.4/../../../../pic32mx/lib\libc.a(_fputc_simple.o) (_flsbuf)
C:/Program Files/Microchip/mplabc32/v1.12/bin/../lib/gcc/pic32mx/3.4.4/../../../../pic32mx/lib\libc.a(_mon_putc.o)
                              C:/Program Files/Microchip/mplabc32/v1.12/bin/../lib/gcc/pic32mx/3.4.4/../../../../pic32mx/lib\libc.a(write.o) (_mon_putc)
C:/Program Files/Microchip/mplabc32/v1.12/bin/../lib/gcc/pic32mx/3.4.4/../../../../pic32mx/lib\libc.a(c32_uart.o)
                              C:/Program Files/Microchip/mplabc32/v1.12/bin/../lib/gcc/pic32mx/3.4.4/../../../../pic32mx/lib\libc.a(_mon_putc.o) (__C32_UART)
C:/Program Files/Microchip/mplabc32/v1.12/bin/../lib/gcc/pic32mx/3.4.4/../../../../pic32mx/lib\libmchp_peripheral.a(open_core_timer_lib.o)
                              output_pic32_ssd1963\DisplayDriver.o (OpenCoreTimer)
C:/Program Files/Microchip/mplabc32/v1.12/bin/../lib/gcc/pic32mx/3.4.4/../../../../pic32mx/lib\libmchp_peripheral_32MX360F512L.a(pcache.o)
                              output_pic32_ssd1963\Application.o (CheKseg0CacheOn)
C:/Program Files/Microchip/mplabc32/v1.12/bin/../lib/gcc/pic32mx/3.4.4/../../../../pic32mx/lib\libmchp_peripheral_32MX360F512L.a(int_disable_interrupts_lib.o)
                              output_pic32_ssd1963\Application.o (INTDisableInterrupts)
C:/Program Files/Microchip/mplabc32/v1.12/bin/../lib/gcc/pic32mx/3.4.4/../../../../pic32mx/lib\libmchp_peripheral_32MX360F512L.a(int_restore_interrupts_lib.o)
                              output_pic32_ssd1963\Application.o (INTRestoreInterrupts)
C:/Program Files/Microchip/mplabc32/v1.12/bin/../lib/gcc/pic32mx/3.4.4/../../../../pic32mx/lib\libmchp_peripheral_32MX360F512L.a(int_enable_mv_int_lib.o)
                              output_pic32_ssd1963\Application.o (INTEnableSystemMultiVectoredInt)
C:/Program Files/Microchip/mplabc32/v1.12/bin/../lib/gcc/pic32mx/3.4.4/../../../../pic32mx/lib\libmchp_peripheral_32MX360F512L.a(spi_getc_spi2_lib_legacy.o)
                              output_pic32_ssd1963\SD-SPI.o (getcSPI2)
C:/Program Files/Microchip/mplabc32/v1.12/bin/../lib/gcc/pic32mx/3.4.4/../../../../pic32mx/lib\libmchp_peripheral_32MX360F512L.a(spi_open_spi2_lib_legacy.o)
                              output_pic32_ssd1963\SD-SPI.o (OpenSPI2)
C:/Program Files/Microchip/mplabc32/v1.12/bin/../lib/gcc/pic32mx/3.4.4/../../../../pic32mx/lib\libmchp_peripheral_32MX360F512L.a(spi_brg_tbl_lib_legacy.o)
                              C:/Program Files/Microchip/mplabc32/v1.12/bin/../lib/gcc/pic32mx/3.4.4/../../../../pic32mx/lib\libmchp_peripheral_32MX360F512L.a(spi_open_spi2_lib_legacy.o) (_SpiBrgConvTbl)
C:/Program Files/Microchip/mplabc32/v1.12/bin/../lib/gcc/pic32mx/3.4.4/../../../../pic32mx/lib\libmchp_peripheral_32MX360F512L.a(int_enable_interrupts_lib.o)
                              C:/Program Files/Microchip/mplabc32/v1.12/bin/../lib/gcc/pic32mx/3.4.4/../../../../pic32mx/lib\libmchp_peripheral_32MX360F512L.a(int_enable_mv_int_lib.o) (INTEnableInterrupts)
C:/Program Files/Microchip/mplabc32/v1.12/bin/../lib/gcc/pic32mx/3.4.4/../../../../pic32mx/lib\libc.a(doprnt_cdnopsuxX.eo)
                              (_vfprintf_cdnopsuxX)
C:/Program Files/Microchip/mplabc32/v1.12/bin/../lib/gcc/pic32mx/3.4.4\libgcc.a(_udivdi3.o)
                              C:/Program Files/Microchip/mplabc32/v1.12/bin/../lib/gcc/pic32mx/3.4.4/../../../../pic32mx/lib\libc.a(doprnt_cdnopuxX.eo) (__udivdi3)
C:/Program Files/Microchip/mplabc32/v1.12/bin/../lib/gcc/pic32mx/3.4.4\libgcc.a(_umoddi3.o)
                              C:/Program Files/Microchip/mplabc32/v1.12/bin/../lib/gcc/pic32mx/3.4.4/../../../../pic32mx/lib\libc.a(doprnt_cdnopuxX.eo) (__umoddi3)

Allocating common symbols
Common symbol       size              file

_cursorY            0x2               output_pic32_ssd1963\Primitive.o
gDataBuffer         0x200             output_pic32_ssd1963\FSIO.o
_activePage         0x1               output_pic32_ssd1963\DisplayDriver.o
IMG_wWidth          0x2               output_pic32_ssd1963\ImageDecoder.o
IMG_bAlignCenter    0x1               output_pic32_ssd1963\ImageDecoder.o
gFileSlotOpen       0x3               output_pic32_ssd1963\FSIO.o
IMG_wStartX         0x2               output_pic32_ssd1963\ImageDecoder.o
gTimeCrtMS          0x1               output_pic32_ssd1963\FSIO.o
MDD_SDSPI_finalLBA  0x4               output_pic32_ssd1963\SD-SPI.o
_fontOrientation    0x1               output_pic32_ssd1963\Primitive.o
_fontFirstChar      0x2               output_pic32_ssd1963\Primitive.o
cwd                 0x3c              output_pic32_ssd1963\FSIO.o
IMG_wHeight         0x2               output_pic32_ssd1963\ImageDecoder.o
defaultString       0xd               output_pic32_ssd1963\FSIO.o
IMG_bDownScalingFactor
                    0x1               output_pic32_ssd1963\ImageDecoder.o
_sibuf              0x20              C:/Program Files/Microchip/mplabc32/v1.12/bin/../lib/gcc/pic32mx/3.4.4/../../../../pic32mx/lib\libc.a(_iob.o)
tempCWDobj          0x3c              output_pic32_ssd1963\FSIO.o
IMG_wStartY         0x2               output_pic32_ssd1963\ImageDecoder.o
_clipRgn            0x2               output_pic32_ssd1963\DisplayDriver.o
_fontHeight         0x2               output_pic32_ssd1963\Primitive.o
gMediaSectorSize    0x2               output_pic32_ssd1963\SD-SPI.o
IMG_wImageWidth     0x2               output_pic32_ssd1963\ImageDecoder.o
IMG_wImageHeight    0x2               output_pic32_ssd1963\ImageDecoder.o
_cursorX            0x2               output_pic32_ssd1963\Primitive.o
_fontLastChar       0x2               output_pic32_ssd1963\Primitive.o
_font               0x4               output_pic32_ssd1963\Primitive.o
_visualPage         0x1               output_pic32_ssd1963\DisplayDriver.o
_lineType           0x2               output_pic32_ssd1963\Primitive.o
gFATBuffer          0x200             output_pic32_ssd1963\FSIO.o
gTimeCrtTime        0x2               output_pic32_ssd1963\FSIO.o
gFileArray          0xb4              output_pic32_ssd1963\FSIO.o
FatRootDirClusterValue
                    0x4               output_pic32_ssd1963\FSIO.o
gDiskData           0x26              output_pic32_ssd1963\FSIO.o
_clipRight          0x2               output_pic32_ssd1963\DisplayDriver.o
gTimeWrtDate        0x2               output_pic32_ssd1963\FSIO.o
_outdone            0x1               C:/Program Files/Microchip/mplabc32/v1.12/bin/../lib/gcc/pic32mx/3.4.4/../../../../pic32mx/lib\libc.a(_iob.o)
IMG_blAbortImageDecoding
                    0x1               output_pic32_ssd1963\ImageDecoder.o
_clipBottom         0x2               output_pic32_ssd1963\DisplayDriver.o
gTimeCrtDate        0x2               output_pic32_ssd1963\FSIO.o
_clipTop            0x2               output_pic32_ssd1963\DisplayDriver.o
_color              0x2               output_pic32_ssd1963\DisplayDriver.o
TempClusterCalc     0x4               output_pic32_ssd1963\FSIO.o
_clipLeft           0x2               output_pic32_ssd1963\DisplayDriver.o
dirCleared          0x1               output_pic32_ssd1963\FSIO.o
gFileTemp           0x3c              output_pic32_ssd1963\FSIO.o
IMG_pLoopCallbackFn
                    0x4               output_pic32_ssd1963\ImageDecoder.o
defaultArray        0xa               output_pic32_ssd1963\FSIO.o
_lineThickness      0x1               output_pic32_ssd1963\Primitive.o
gSDMode             0x1               output_pic32_ssd1963\SD-SPI.o
gTimeAccDate        0x2               output_pic32_ssd1963\FSIO.o
FSerrno             0x1               output_pic32_ssd1963\FSIO.o
_sobuf              0x20              C:/Program Files/Microchip/mplabc32/v1.12/bin/../lib/gcc/pic32mx/3.4.4/../../../../pic32mx/lib\libc.a(_iob.o)
gTimeWrtTime        0x2               output_pic32_ssd1963\FSIO.o

Microchip PIC32 Memory-Usage Report

kseg0 Program-Memory Usage
section                    address  length [bytes]      (dec)  Description
-------                 ----------  -------------------------  -----------
.text                   0x9d000000        0x11d20       72992  Application's executable code 
.rodata                 0x9d011d20         0x25a4        9636  Read-only constant data 
.eh_frame               0x9d0142c4           0x50          80  Stack unwind info 
.data                   0x9d014314           0xa0         160  Data-initialization template 
.sdata                  0x9d0143b4           0x14          20  Small data-initialization template 
      Total kseg0_program_mem used  :     0x143c8       82888  15.8% of 0x80000

kseg0 Boot-Memory Usage
section                    address  length [bytes]      (dec)  Description
-------                 ----------  -------------------------  -----------
.startup                0x9fc00490          0x1e0         480  C startup code 
         Total kseg0_boot_mem used  :       0x1e0         480  19.9% of 0x970

Exception-Memory Usage 
section                    address  length [bytes]      (dec)  Description
-------                 ----------  -------------------------  -----------
.app_excpt              0x9fc01180           0x10          16  General-Exception handler 
          Total exception_mem used  :        0x10          16  0.4% of 0x1000

kseg1 Boot-Memory Usage
section                    address  length [bytes]      (dec)  Description
-------                 ----------  -------------------------  -----------
.reset                  0xbfc00000           0x10          16  Reset handler 
.bev_excpt              0xbfc00380           0x10          16  BEV-Exception handler 
         Total kseg1_boot_mem used  :        0x20          32  2.7% of 0x490
        --------------------------------------------------------------------------
         Total Program Memory used  :     0x145d8       83416  15.7% of 0x81e00
        --------------------------------------------------------------------------


kseg1 Data-Memory Usage
section                    address  length [bytes]      (dec)  Description
-------                 ----------  -------------------------  -----------
.data                   0xa0000000           0xa0         160  Initialized data 
.sdata                  0xa00000a0           0x14          20  Small initialized data 
.sbss                   0xa00000b4           0x79         121  Small uninitialized data 
.bss                    0xa0000130          0x5ec        1516  Uninitialized data 
.heap                   0xa0000720         0x2000        8192  Dynamic Memory heap 
.stack                  0xa0002720          0x800        2048  Minimum space reserved for stack 
         Total kseg1_data_mem used  :      0x2f19       12057  36.8% of 0x8000
        --------------------------------------------------------------------------
            Total Data Memory used  :      0x2f19       12057  36.8% of 0x8000
        --------------------------------------------------------------------------

Discarded input sections

 .data          0x00000000        0x0 C:/Program Files/Microchip/mplabc32/v1.12/bin/../lib/gcc/pic32mx/3.4.4/../../../../pic32mx/lib/crt0.o
 .bss           0x00000000        0x0 C:/Program Files/Microchip/mplabc32/v1.12/bin/../lib/gcc/pic32mx/3.4.4/../../../../pic32mx/lib/crt0.o
 .reginfo       0x00000000       0x18 C:/Program Files/Microchip/mplabc32/v1.12/bin/../lib/gcc/pic32mx/3.4.4/../../../../pic32mx/lib/crt0.o
 .pdr           0x00000000       0xa0 C:/Program Files/Microchip/mplabc32/v1.12/bin/../lib/gcc/pic32mx/3.4.4/../../../../pic32mx/lib/crt0.o
 .data          0x00000000        0x0 output_pic32_ssd1963\Application.o
 .bss           0x00000000        0x0 output_pic32_ssd1963\Application.o
 .reginfo       0x00000000       0x18 output_pic32_ssd1963\Application.o
 .pdr           0x00000000       0x40 output_pic32_ssd1963\Application.o
 .data          0x00000000        0x0 output_pic32_ssd1963\Primitive.o
 .bss           0x00000000        0x0 output_pic32_ssd1963\Primitive.o
 .reginfo       0x00000000       0x18 output_pic32_ssd1963\Primitive.o
 .pdr           0x00000000      0x1c0 output_pic32_ssd1963\Primitive.o
 .text          0x00000000        0x0 output_pic32_ssd1963\GOLFontDefault.o
 .data          0x00000000        0x0 output_pic32_ssd1963\GOLFontDefault.o
 .bss           0x00000000        0x0 output_pic32_ssd1963\GOLFontDefault.o
 .reginfo       0x00000000       0x18 output_pic32_ssd1963\GOLFontDefault.o
 .pdr           0x00000000        0x0 output_pic32_ssd1963\GOLFontDefault.o
 .data          0x00000000        0x0 output_pic32_ssd1963\JpegDecoder.o
 .bss           0x00000000        0x0 output_pic32_ssd1963\JpegDecoder.o
 .reginfo       0x00000000       0x18 output_pic32_ssd1963\JpegDecoder.o
 .pdr           0x00000000      0x1c0 output_pic32_ssd1963\JpegDecoder.o
 .data          0x00000000        0x0 output_pic32_ssd1963\BmpDecoder.o
 .bss           0x00000000        0x0 output_pic32_ssd1963\BmpDecoder.o
 .reginfo       0x00000000       0x18 output_pic32_ssd1963\BmpDecoder.o
 .pdr           0x00000000       0x60 output_pic32_ssd1963\BmpDecoder.o
 .data          0x00000000        0x0 output_pic32_ssd1963\GifDecoder.o
 .bss           0x00000000        0x0 output_pic32_ssd1963\GifDecoder.o
 .reginfo       0x00000000       0x18 output_pic32_ssd1963\GifDecoder.o
 .pdr           0x00000000      0x1e0 output_pic32_ssd1963\GifDecoder.o
 .data          0x00000000        0x0 output_pic32_ssd1963\ImageDecoder.o
 .bss           0x00000000        0x0 output_pic32_ssd1963\ImageDecoder.o
 .reginfo       0x00000000       0x18 output_pic32_ssd1963\ImageDecoder.o
 .pdr           0x00000000       0x80 output_pic32_ssd1963\ImageDecoder.o
 .data          0x00000000        0x0 output_pic32_ssd1963\jidctint.o
 .bss           0x00000000        0x0 output_pic32_ssd1963\jidctint.o
 .reginfo       0x00000000       0x18 output_pic32_ssd1963\jidctint.o
 .pdr           0x00000000       0x20 output_pic32_ssd1963\jidctint.o
 .data          0x00000000        0x0 output_pic32_ssd1963\DisplayDriver.o
 .bss           0x00000000        0x0 output_pic32_ssd1963\DisplayDriver.o
 .reginfo       0x00000000       0x18 output_pic32_ssd1963\DisplayDriver.o
 .pdr           0x00000000      0x300 output_pic32_ssd1963\DisplayDriver.o
 .data          0x00000000        0x0 output_pic32_ssd1963\SD-SPI.o
 .bss           0x00000000        0x0 output_pic32_ssd1963\SD-SPI.o
 .reginfo       0x00000000       0x18 output_pic32_ssd1963\SD-SPI.o
 .pdr           0x00000000      0x1e0 output_pic32_ssd1963\SD-SPI.o
 .data          0x00000000        0x0 output_pic32_ssd1963\FSIO.o
 .bss           0x00000000        0x0 output_pic32_ssd1963\FSIO.o
 .reginfo       0x00000000       0x18 output_pic32_ssd1963\FSIO.o
 .pdr           0x00000000      0x7a0 output_pic32_ssd1963\FSIO.o
 .text          0x00000000        0x0 output_pic32_ssd1963\GOLMediumlFont.o
 .data          0x00000000        0x0 output_pic32_ssd1963\GOLMediumlFont.o
 .bss           0x00000000        0x0 output_pic32_ssd1963\GOLMediumlFont.o
 .reginfo       0x00000000       0x18 output_pic32_ssd1963\GOLMediumlFont.o
 .pdr           0x00000000        0x0 output_pic32_ssd1963\GOLMediumlFont.o
 .rodata        0x00000000      0xae4 output_pic32_ssd1963\GOLMediumlFont.o
 .text          0x00000000        0x0 output_pic32_ssd1963\GOLSmallFont.o
 .data          0x00000000        0x0 output_pic32_ssd1963\GOLSmallFont.o
 .bss           0x00000000        0x0 output_pic32_ssd1963\GOLSmallFont.o
 .reginfo       0x00000000       0x18 output_pic32_ssd1963\GOLSmallFont.o
 .pdr           0x00000000        0x0 output_pic32_ssd1963\GOLSmallFont.o
 .data          0x00000000        0x0 C:/Program Files/Microchip/mplabc32/v1.12/bin/../lib/gcc/pic32mx/3.4.4/../../../../pic32mx/lib\libc.a(memset.o)
 .bss           0x00000000        0x0 C:/Program Files/Microchip/mplabc32/v1.12/bin/../lib/gcc/pic32mx/3.4.4/../../../../pic32mx/lib\libc.a(memset.o)
 .reginfo       0x00000000       0x18 C:/Program Files/Microchip/mplabc32/v1.12/bin/../lib/gcc/pic32mx/3.4.4/../../../../pic32mx/lib\libc.a(memset.o)
 .pdr           0x00000000       0x20 C:/Program Files/Microchip/mplabc32/v1.12/bin/../lib/gcc/pic32mx/3.4.4/../../../../pic32mx/lib\libc.a(memset.o)
 .data          0x00000000        0x0 C:/Program Files/Microchip/mplabc32/v1.12/bin/../lib/gcc/pic32mx/3.4.4/../../../../pic32mx/lib\libc.a(strcpy.o)
 .bss           0x00000000        0x0 C:/Program Files/Microchip/mplabc32/v1.12/bin/../lib/gcc/pic32mx/3.4.4/../../../../pic32mx/lib\libc.a(strcpy.o)
 .reginfo       0x00000000       0x18 C:/Program Files/Microchip/mplabc32/v1.12/bin/../lib/gcc/pic32mx/3.4.4/../../../../pic32mx/lib\libc.a(strcpy.o)
 .pdr           0x00000000       0x20 C:/Program Files/Microchip/mplabc32/v1.12/bin/../lib/gcc/pic32mx/3.4.4/../../../../pic32mx/lib\libc.a(strcpy.o)
 .data          0x00000000        0x0 C:/Program Files/Microchip/mplabc32/v1.12/bin/../lib/gcc/pic32mx/3.4.4/../../../../pic32mx/lib\libc.a(strlen.o)
 .bss           0x00000000        0x0 C:/Program Files/Microchip/mplabc32/v1.12/bin/../lib/gcc/pic32mx/3.4.4/../../../../pic32mx/lib\libc.a(strlen.o)
 .reginfo       0x00000000       0x18 C:/Program Files/Microchip/mplabc32/v1.12/bin/../lib/gcc/pic32mx/3.4.4/../../../../pic32mx/lib\libc.a(strlen.o)
 .pdr           0x00000000       0x20 C:/Program Files/Microchip/mplabc32/v1.12/bin/../lib/gcc/pic32mx/3.4.4/../../../../pic32mx/lib\libc.a(strlen.o)
 .text          0x00000000        0x0 C:/Program Files/Microchip/mplabc32/v1.12/bin/../lib/gcc/pic32mx/3.4.4/../../../../pic32mx/lib\libc.a(general-exception.o)
 .data          0x00000000        0x0 C:/Program Files/Microchip/mplabc32/v1.12/bin/../lib/gcc/pic32mx/3.4.4/../../../../pic32mx/lib\libc.a(general-exception.o)
 .bss           0x00000000        0x0 C:/Program Files/Microchip/mplabc32/v1.12/bin/../lib/gcc/pic32mx/3.4.4/../../../../pic32mx/lib\libc.a(general-exception.o)
 .reginfo       0x00000000       0x18 C:/Program Files/Microchip/mplabc32/v1.12/bin/../lib/gcc/pic32mx/3.4.4/../../../../pic32mx/lib\libc.a(general-exception.o)
 .pdr           0x00000000       0x20 C:/Program Files/Microchip/mplabc32/v1.12/bin/../lib/gcc/pic32mx/3.4.4/../../../../pic32mx/lib\libc.a(general-exception.o)
 .text          0x00000000        0x0 C:/Program Files/Microchip/mplabc32/v1.12/bin/../lib/gcc/pic32mx/3.4.4/../../../../pic32mx/lib\libc.a(ctypef.o)
 .data          0x00000000        0x0 C:/Program Files/Microchip/mplabc32/v1.12/bin/../lib/gcc/pic32mx/3.4.4/../../../../pic32mx/lib\libc.a(ctypef.o)
 .bss           0x00000000        0x0 C:/Program Files/Microchip/mplabc32/v1.12/bin/../lib/gcc/pic32mx/3.4.4/../../../../pic32mx/lib\libc.a(ctypef.o)
 .reginfo       0x00000000       0x18 C:/Program Files/Microchip/mplabc32/v1.12/bin/../lib/gcc/pic32mx/3.4.4/../../../../pic32mx/lib\libc.a(ctypef.o)
 .pdr           0x00000000      0x220 C:/Program Files/Microchip/mplabc32/v1.12/bin/../lib/gcc/pic32mx/3.4.4/../../../../pic32mx/lib\libc.a(ctypef.o)
 .text.isalnum  0x00000000       0x18 C:/Program Files/Microchip/mplabc32/v1.12/bin/../lib/gcc/pic32mx/3.4.4/../../../../pic32mx/lib\libc.a(ctypef.o)
 .text.isalpha  0x00000000       0x18 C:/Program Files/Microchip/mplabc32/v1.12/bin/../lib/gcc/pic32mx/3.4.4/../../../../pic32mx/lib\libc.a(ctypef.o)
 .text.isascii  0x00000000        0x8 C:/Program Files/Microchip/mplabc32/v1.12/bin/../lib/gcc/pic32mx/3.4.4/../../../../pic32mx/lib\libc.a(ctypef.o)
 .text.iscntrl  0x00000000       0x18 C:/Program Files/Microchip/mplabc32/v1.12/bin/../lib/gcc/pic32mx/3.4.4/../../../../pic32mx/lib\libc.a(ctypef.o)
 .text.isdigit  0x00000000       0x18 C:/Program Files/Microchip/mplabc32/v1.12/bin/../lib/gcc/pic32mx/3.4.4/../../../../pic32mx/lib\libc.a(ctypef.o)
 .text.isgraph  0x00000000       0x18 C:/Program Files/Microchip/mplabc32/v1.12/bin/../lib/gcc/pic32mx/3.4.4/../../../../pic32mx/lib\libc.a(ctypef.o)
 .text.islower  0x00000000       0x18 C:/Program Files/Microchip/mplabc32/v1.12/bin/../lib/gcc/pic32mx/3.4.4/../../../../pic32mx/lib\libc.a(ctypef.o)
 .text.isprint  0x00000000       0x18 C:/Program Files/Microchip/mplabc32/v1.12/bin/../lib/gcc/pic32mx/3.4.4/../../../../pic32mx/lib\libc.a(ctypef.o)
 .text.ispunct  0x00000000       0x18 C:/Program Files/Microchip/mplabc32/v1.12/bin/../lib/gcc/pic32mx/3.4.4/../../../../pic32mx/lib\libc.a(ctypef.o)
 .text.isspace  0x00000000       0x18 C:/Program Files/Microchip/mplabc32/v1.12/bin/../lib/gcc/pic32mx/3.4.4/../../../../pic32mx/lib\libc.a(ctypef.o)
 .text.isupper  0x00000000       0x18 C:/Program Files/Microchip/mplabc32/v1.12/bin/../lib/gcc/pic32mx/3.4.4/../../../../pic32mx/lib\libc.a(ctypef.o)
 .text.isxdigit
                0x00000000       0x18 C:/Program Files/Microchip/mplabc32/v1.12/bin/../lib/gcc/pic32mx/3.4.4/../../../../pic32mx/lib\libc.a(ctypef.o)
 .text.toascii  0x00000000        0x8 C:/Program Files/Microchip/mplabc32/v1.12/bin/../lib/gcc/pic32mx/3.4.4/../../../../pic32mx/lib\libc.a(ctypef.o)
 .text._tolower
                0x00000000        0x8 C:/Program Files/Microchip/mplabc32/v1.12/bin/../lib/gcc/pic32mx/3.4.4/../../../../pic32mx/lib\libc.a(ctypef.o)
 .text._toupper
                0x00000000        0x8 C:/Program Files/Microchip/mplabc32/v1.12/bin/../lib/gcc/pic32mx/3.4.4/../../../../pic32mx/lib\libc.a(ctypef.o)
 .text          0x00000000        0x0 C:/Program Files/Microchip/mplabc32/v1.12/bin/../lib/gcc/pic32mx/3.4.4/../../../../pic32mx/lib\libc.a(puts.o)
 .data          0x00000000        0x0 C:/Program Files/Microchip/mplabc32/v1.12/bin/../lib/gcc/pic32mx/3.4.4/../../../../pic32mx/lib\libc.a(puts.o)
 .bss           0x00000000        0x0 C:/Program Files/Microchip/mplabc32/v1.12/bin/../lib/gcc/pic32mx/3.4.4/../../../../pic32mx/lib\libc.a(puts.o)
 .reginfo       0x00000000       0x18 C:/Program Files/Microchip/mplabc32/v1.12/bin/../lib/gcc/pic32mx/3.4.4/../../../../pic32mx/lib\libc.a(puts.o)
 .pdr           0x00000000       0x40 C:/Program Files/Microchip/mplabc32/v1.12/bin/../lib/gcc/pic32mx/3.4.4/../../../../pic32mx/lib\libc.a(puts.o)
 .text          0x00000000        0x0 C:/Program Files/Microchip/mplabc32/v1.12/bin/../lib/gcc/pic32mx/3.4.4/../../../../pic32mx/lib\libc.a(strchr.o)
 .data          0x00000000        0x0 C:/Program Files/Microchip/mplabc32/v1.12/bin/../lib/gcc/pic32mx/3.4.4/../../../../pic32mx/lib\libc.a(strchr.o)
 .bss           0x00000000        0x0 C:/Program Files/Microchip/mplabc32/v1.12/bin/../lib/gcc/pic32mx/3.4.4/../../../../pic32mx/lib\libc.a(strchr.o)
 .reginfo       0x00000000       0x18 C:/Program Files/Microchip/mplabc32/v1.12/bin/../lib/gcc/pic32mx/3.4.4/../../../../pic32mx/lib\libc.a(strchr.o)
 .pdr           0x00000000       0x20 C:/Program Files/Microchip/mplabc32/v1.12/bin/../lib/gcc/pic32mx/3.4.4/../../../../pic32mx/lib\libc.a(strchr.o)
 .text          0x00000000        0x0 C:/Program Files/Microchip/mplabc32/v1.12/bin/../lib/gcc/pic32mx/3.4.4/../../../../pic32mx/lib\libc.a(strncpy.o)
 .data          0x00000000        0x0 C:/Program Files/Microchip/mplabc32/v1.12/bin/../lib/gcc/pic32mx/3.4.4/../../../../pic32mx/lib\libc.a(strncpy.o)
 .bss           0x00000000        0x0 C:/Program Files/Microchip/mplabc32/v1.12/bin/../lib/gcc/pic32mx/3.4.4/../../../../pic32mx/lib\libc.a(strncpy.o)
 .reginfo       0x00000000       0x18 C:/Program Files/Microchip/mplabc32/v1.12/bin/../lib/gcc/pic32mx/3.4.4/../../../../pic32mx/lib\libc.a(strncpy.o)
 .pdr           0x00000000       0x20 C:/Program Files/Microchip/mplabc32/v1.12/bin/../lib/gcc/pic32mx/3.4.4/../../../../pic32mx/lib\libc.a(strncpy.o)
 .text          0x00000000        0x0 C:/Program Files/Microchip/mplabc32/v1.12/bin/../lib/gcc/pic32mx/3.4.4/../../../../pic32mx/lib\libc.a(printf_cdnopuxX.eo)
 .data          0x00000000        0x0 C:/Program Files/Microchip/mplabc32/v1.12/bin/../lib/gcc/pic32mx/3.4.4/../../../../pic32mx/lib\libc.a(printf_cdnopuxX.eo)
 .bss           0x00000000        0x0 C:/Program Files/Microchip/mplabc32/v1.12/bin/../lib/gcc/pic32mx/3.4.4/../../../../pic32mx/lib\libc.a(printf_cdnopuxX.eo)
 .reginfo       0x00000000       0x18 C:/Program Files/Microchip/mplabc32/v1.12/bin/../lib/gcc/pic32mx/3.4.4/../../../../pic32mx/lib\libc.a(printf_cdnopuxX.eo)
 .pdr           0x00000000       0x20 C:/Program Files/Microchip/mplabc32/v1.12/bin/../lib/gcc/pic32mx/3.4.4/../../../../pic32mx/lib\libc.a(printf_cdnopuxX.eo)
 .text          0x00000000        0x0 C:/Program Files/Microchip/mplabc32/v1.12/bin/../lib/gcc/pic32mx/3.4.4/../../../../pic32mx/lib\libc.a(sprintf_s.eo)
 .data          0x00000000        0x0 C:/Program Files/Microchip/mplabc32/v1.12/bin/../lib/gcc/pic32mx/3.4.4/../../../../pic32mx/lib\libc.a(sprintf_s.eo)
 .bss           0x00000000        0x0 C:/Program Files/Microchip/mplabc32/v1.12/bin/../lib/gcc/pic32mx/3.4.4/../../../../pic32mx/lib\libc.a(sprintf_s.eo)
 .reginfo       0x00000000       0x18 C:/Program Files/Microchip/mplabc32/v1.12/bin/../lib/gcc/pic32mx/3.4.4/../../../../pic32mx/lib\libc.a(sprintf_s.eo)
 .pdr           0x00000000       0x20 C:/Program Files/Microchip/mplabc32/v1.12/bin/../lib/gcc/pic32mx/3.4.4/../../../../pic32mx/lib\libc.a(sprintf_s.eo)
 .text          0x00000000        0x0 C:/Program Files/Microchip/mplabc32/v1.12/bin/../lib/gcc/pic32mx/3.4.4/../../../../pic32mx/lib\libc.a(default-general-exception-handler.o)
 .data          0x00000000        0x0 C:/Program Files/Microchip/mplabc32/v1.12/bin/../lib/gcc/pic32mx/3.4.4/../../../../pic32mx/lib\libc.a(default-general-exception-handler.o)
 .bss           0x00000000        0x0 C:/Program Files/Microchip/mplabc32/v1.12/bin/../lib/gcc/pic32mx/3.4.4/../../../../pic32mx/lib\libc.a(default-general-exception-handler.o)
 .reginfo       0x00000000       0x18 C:/Program Files/Microchip/mplabc32/v1.12/bin/../lib/gcc/pic32mx/3.4.4/../../../../pic32mx/lib\libc.a(default-general-exception-handler.o)
 .pdr           0x00000000       0x20 C:/Program Files/Microchip/mplabc32/v1.12/bin/../lib/gcc/pic32mx/3.4.4/../../../../pic32mx/lib\libc.a(default-general-exception-handler.o)
 .text          0x00000000        0x0 C:/Program Files/Microchip/mplabc32/v1.12/bin/../lib/gcc/pic32mx/3.4.4/../../../../pic32mx/lib\libc.a(default-bootstrap-exception-handler.o)
 .data          0x00000000        0x0 C:/Program Files/Microchip/mplabc32/v1.12/bin/../lib/gcc/pic32mx/3.4.4/../../../../pic32mx/lib\libc.a(default-bootstrap-exception-handler.o)
 .bss           0x00000000        0x0 C:/Program Files/Microchip/mplabc32/v1.12/bin/../lib/gcc/pic32mx/3.4.4/../../../../pic32mx/lib\libc.a(default-bootstrap-exception-handler.o)
 .reginfo       0x00000000       0x18 C:/Program Files/Microchip/mplabc32/v1.12/bin/../lib/gcc/pic32mx/3.4.4/../../../../pic32mx/lib\libc.a(default-bootstrap-exception-handler.o)
 .pdr           0x00000000       0x20 C:/Program Files/Microchip/mplabc32/v1.12/bin/../lib/gcc/pic32mx/3.4.4/../../../../pic32mx/lib\libc.a(default-bootstrap-exception-handler.o)
 .text          0x00000000        0x0 C:/Program Files/Microchip/mplabc32/v1.12/bin/../lib/gcc/pic32mx/3.4.4/../../../../pic32mx/lib\libc.a(default-on-reset.o)
 .data          0x00000000        0x0 C:/Program Files/Microchip/mplabc32/v1.12/bin/../lib/gcc/pic32mx/3.4.4/../../../../pic32mx/lib\libc.a(default-on-reset.o)
 .bss           0x00000000        0x0 C:/Program Files/Microchip/mplabc32/v1.12/bin/../lib/gcc/pic32mx/3.4.4/../../../../pic32mx/lib\libc.a(default-on-reset.o)
 .reginfo       0x00000000       0x18 C:/Program Files/Microchip/mplabc32/v1.12/bin/../lib/gcc/pic32mx/3.4.4/../../../../pic32mx/lib\libc.a(default-on-reset.o)
 .pdr           0x00000000       0x20 C:/Program Files/Microchip/mplabc32/v1.12/bin/../lib/gcc/pic32mx/3.4.4/../../../../pic32mx/lib\libc.a(default-on-reset.o)
 .text          0x00000000        0x0 C:/Program Files/Microchip/mplabc32/v1.12/bin/../lib/gcc/pic32mx/3.4.4/../../../../pic32mx/lib\libc.a(default-on-bootstrap.o)
 .data          0x00000000        0x0 C:/Program Files/Microchip/mplabc32/v1.12/bin/../lib/gcc/pic32mx/3.4.4/../../../../pic32mx/lib\libc.a(default-on-bootstrap.o)
 .bss           0x00000000        0x0 C:/Program Files/Microchip/mplabc32/v1.12/bin/../lib/gcc/pic32mx/3.4.4/../../../../pic32mx/lib\libc.a(default-on-bootstrap.o)
 .reginfo       0x00000000       0x18 C:/Program Files/Microchip/mplabc32/v1.12/bin/../lib/gcc/pic32mx/3.4.4/../../../../pic32mx/lib\libc.a(default-on-bootstrap.o)
 .pdr           0x00000000       0x20 C:/Program Files/Microchip/mplabc32/v1.12/bin/../lib/gcc/pic32mx/3.4.4/../../../../pic32mx/lib\libc.a(default-on-bootstrap.o)
 .data          0x00000000        0x0 C:/Program Files/Microchip/mplabc32/v1.12/bin/../lib/gcc/pic32mx/3.4.4/../../../../pic32mx/lib\libc.a(default-nmi-handler.o)
 .bss           0x00000000        0x0 C:/Program Files/Microchip/mplabc32/v1.12/bin/../lib/gcc/pic32mx/3.4.4/../../../../pic32mx/lib\libc.a(default-nmi-handler.o)
 .reginfo       0x00000000       0x18 C:/Program Files/Microchip/mplabc32/v1.12/bin/../lib/gcc/pic32mx/3.4.4/../../../../pic32mx/lib\libc.a(default-nmi-handler.o)
 .pdr           0x00000000       0x20 C:/Program Files/Microchip/mplabc32/v1.12/bin/../lib/gcc/pic32mx/3.4.4/../../../../pic32mx/lib\libc.a(default-nmi-handler.o)
 .text          0x00000000        0x0 C:/Program Files/Microchip/mplabc32/v1.12/bin/../lib/gcc/pic32mx/3.4.4/../../../../pic32mx/lib\libc.a(_iob.o)
 .bss           0x00000000        0x0 C:/Program Files/Microchip/mplabc32/v1.12/bin/../lib/gcc/pic32mx/3.4.4/../../../../pic32mx/lib\libc.a(_iob.o)
 .reginfo       0x00000000       0x18 C:/Program Files/Microchip/mplabc32/v1.12/bin/../lib/gcc/pic32mx/3.4.4/../../../../pic32mx/lib\libc.a(_iob.o)
 .pdr           0x00000000        0x0 C:/Program Files/Microchip/mplabc32/v1.12/bin/../lib/gcc/pic32mx/3.4.4/../../../../pic32mx/lib\libc.a(_iob.o)
 .sdata         0x00000000        0x4 C:/Program Files/Microchip/mplabc32/v1.12/bin/../lib/gcc/pic32mx/3.4.4/../../../../pic32mx/lib\libc.a(_iob.o)
 .text          0x00000000        0x0 C:/Program Files/Microchip/mplabc32/v1.12/bin/../lib/gcc/pic32mx/3.4.4/../../../../pic32mx/lib\libc.a(_fputc_simple.o)
 .data          0x00000000        0x0 C:/Program Files/Microchip/mplabc32/v1.12/bin/../lib/gcc/pic32mx/3.4.4/../../../../pic32mx/lib\libc.a(_fputc_simple.o)
 .bss           0x00000000        0x0 C:/Program Files/Microchip/mplabc32/v1.12/bin/../lib/gcc/pic32mx/3.4.4/../../../../pic32mx/lib\libc.a(_fputc_simple.o)
 .reginfo       0x00000000       0x18 C:/Program Files/Microchip/mplabc32/v1.12/bin/../lib/gcc/pic32mx/3.4.4/../../../../pic32mx/lib\libc.a(_fputc_simple.o)
 .pdr           0x00000000       0x20 C:/Program Files/Microchip/mplabc32/v1.12/bin/../lib/gcc/pic32mx/3.4.4/../../../../pic32mx/lib\libc.a(_fputc_simple.o)
 .text          0x00000000        0x0 C:/Program Files/Microchip/mplabc32/v1.12/bin/../lib/gcc/pic32mx/3.4.4/../../../../pic32mx/lib\libc.a(ctype.o)
 .data          0x00000000        0x0 C:/Program Files/Microchip/mplabc32/v1.12/bin/../lib/gcc/pic32mx/3.4.4/../../../../pic32mx/lib\libc.a(ctype.o)
 .bss           0x00000000        0x0 C:/Program Files/Microchip/mplabc32/v1.12/bin/../lib/gcc/pic32mx/3.4.4/../../../../pic32mx/lib\libc.a(ctype.o)
 .reginfo       0x00000000       0x18 C:/Program Files/Microchip/mplabc32/v1.12/bin/../lib/gcc/pic32mx/3.4.4/../../../../pic32mx/lib\libc.a(ctype.o)
 .pdr           0x00000000        0x0 C:/Program Files/Microchip/mplabc32/v1.12/bin/../lib/gcc/pic32mx/3.4.4/../../../../pic32mx/lib\libc.a(ctype.o)
 .text          0x00000000        0x0 C:/Program Files/Microchip/mplabc32/v1.12/bin/../lib/gcc/pic32mx/3.4.4/../../../../pic32mx/lib\libc.a(write.o)
 .data          0x00000000        0x0 C:/Program Files/Microchip/mplabc32/v1.12/bin/../lib/gcc/pic32mx/3.4.4/../../../../pic32mx/lib\libc.a(write.o)
 .bss           0x00000000        0x0 C:/Program Files/Microchip/mplabc32/v1.12/bin/../lib/gcc/pic32mx/3.4.4/../../../../pic32mx/lib\libc.a(write.o)
 .reginfo       0x00000000       0x18 C:/Program Files/Microchip/mplabc32/v1.12/bin/../lib/gcc/pic32mx/3.4.4/../../../../pic32mx/lib\libc.a(write.o)
 .pdr           0x00000000       0x20 C:/Program Files/Microchip/mplabc32/v1.12/bin/../lib/gcc/pic32mx/3.4.4/../../../../pic32mx/lib\libc.a(write.o)
 .text          0x00000000        0x0 C:/Program Files/Microchip/mplabc32/v1.12/bin/../lib/gcc/pic32mx/3.4.4/../../../../pic32mx/lib\libc.a(_flsbuf_simple.o)
 .data          0x00000000        0x0 C:/Program Files/Microchip/mplabc32/v1.12/bin/../lib/gcc/pic32mx/3.4.4/../../../../pic32mx/lib\libc.a(_flsbuf_simple.o)
 .bss           0x00000000        0x0 C:/Program Files/Microchip/mplabc32/v1.12/bin/../lib/gcc/pic32mx/3.4.4/../../../../pic32mx/lib\libc.a(_flsbuf_simple.o)
 .reginfo       0x00000000       0x18 C:/Program Files/Microchip/mplabc32/v1.12/bin/../lib/gcc/pic32mx/3.4.4/../../../../pic32mx/lib\libc.a(_flsbuf_simple.o)
 .pdr           0x00000000       0x20 C:/Program Files/Microchip/mplabc32/v1.12/bin/../lib/gcc/pic32mx/3.4.4/../../../../pic32mx/lib\libc.a(_flsbuf_simple.o)
 .text          0x00000000        0x0 C:/Program Files/Microchip/mplabc32/v1.12/bin/../lib/gcc/pic32mx/3.4.4/../../../../pic32mx/lib\libc.a(_mon_putc.o)
 .data          0x00000000        0x0 C:/Program Files/Microchip/mplabc32/v1.12/bin/../lib/gcc/pic32mx/3.4.4/../../../../pic32mx/lib\libc.a(_mon_putc.o)
 .bss           0x00000000        0x0 C:/Program Files/Microchip/mplabc32/v1.12/bin/../lib/gcc/pic32mx/3.4.4/../../../../pic32mx/lib\libc.a(_mon_putc.o)
 .reginfo       0x00000000       0x18 C:/Program Files/Microchip/mplabc32/v1.12/bin/../lib/gcc/pic32mx/3.4.4/../../../../pic32mx/lib\libc.a(_mon_putc.o)
 .pdr           0x00000000       0x20 C:/Program Files/Microchip/mplabc32/v1.12/bin/../lib/gcc/pic32mx/3.4.4/../../../../pic32mx/lib\libc.a(_mon_putc.o)
 .text          0x00000000        0x0 C:/Program Files/Microchip/mplabc32/v1.12/bin/../lib/gcc/pic32mx/3.4.4/../../../../pic32mx/lib\libc.a(c32_uart.o)
 .data          0x00000000        0x0 C:/Program Files/Microchip/mplabc32/v1.12/bin/../lib/gcc/pic32mx/3.4.4/../../../../pic32mx/lib\libc.a(c32_uart.o)
 .bss           0x00000000        0x0 C:/Program Files/Microchip/mplabc32/v1.12/bin/../lib/gcc/pic32mx/3.4.4/../../../../pic32mx/lib\libc.a(c32_uart.o)
 .reginfo       0x00000000       0x18 C:/Program Files/Microchip/mplabc32/v1.12/bin/../lib/gcc/pic32mx/3.4.4/../../../../pic32mx/lib\libc.a(c32_uart.o)
 .pdr           0x00000000        0x0 C:/Program Files/Microchip/mplabc32/v1.12/bin/../lib/gcc/pic32mx/3.4.4/../../../../pic32mx/lib\libc.a(c32_uart.o)
 .text          0x00000000        0x0 C:/Program Files/Microchip/mplabc32/v1.12/bin/../lib/gcc/pic32mx/3.4.4/../../../../pic32mx/lib\libmchp_peripheral.a(open_core_timer_lib.o)
 .data          0x00000000        0x0 C:/Program Files/Microchip/mplabc32/v1.12/bin/../lib/gcc/pic32mx/3.4.4/../../../../pic32mx/lib\libmchp_peripheral.a(open_core_timer_lib.o)
 .bss           0x00000000        0x0 C:/Program Files/Microchip/mplabc32/v1.12/bin/../lib/gcc/pic32mx/3.4.4/../../../../pic32mx/lib\libmchp_peripheral.a(open_core_timer_lib.o)
 .reginfo       0x00000000       0x18 C:/Program Files/Microchip/mplabc32/v1.12/bin/../lib/gcc/pic32mx/3.4.4/../../../../pic32mx/lib\libmchp_peripheral.a(open_core_timer_lib.o)
 .pdr           0x00000000       0x20 C:/Program Files/Microchip/mplabc32/v1.12/bin/../lib/gcc/pic32mx/3.4.4/../../../../pic32mx/lib\libmchp_peripheral.a(open_core_timer_lib.o)
 .text          0x00000000        0x0 C:/Program Files/Microchip/mplabc32/v1.12/bin/../lib/gcc/pic32mx/3.4.4/../../../../pic32mx/lib\libmchp_peripheral_32MX360F512L.a(pcache.o)
 .data          0x00000000        0x0 C:/Program Files/Microchip/mplabc32/v1.12/bin/../lib/gcc/pic32mx/3.4.4/../../../../pic32mx/lib\libmchp_peripheral_32MX360F512L.a(pcache.o)
 .bss           0x00000000        0x0 C:/Program Files/Microchip/mplabc32/v1.12/bin/../lib/gcc/pic32mx/3.4.4/../../../../pic32mx/lib\libmchp_peripheral_32MX360F512L.a(pcache.o)
 .reginfo       0x00000000       0x18 C:/Program Files/Microchip/mplabc32/v1.12/bin/../lib/gcc/pic32mx/3.4.4/../../../../pic32mx/lib\libmchp_peripheral_32MX360F512L.a(pcache.o)
 .pdr           0x00000000       0x40 C:/Program Files/Microchip/mplabc32/v1.12/bin/../lib/gcc/pic32mx/3.4.4/../../../../pic32mx/lib\libmchp_peripheral_32MX360F512L.a(pcache.o)
 .text.CheKseg0CacheOff
                0x00000000       0x18 C:/Program Files/Microchip/mplabc32/v1.12/bin/../lib/gcc/pic32mx/3.4.4/../../../../pic32mx/lib\libmchp_peripheral_32MX360F512L.a(pcache.o)
 .text          0x00000000        0x0 C:/Program Files/Microchip/mplabc32/v1.12/bin/../lib/gcc/pic32mx/3.4.4/../../../../pic32mx/lib\libmchp_peripheral_32MX360F512L.a(int_disable_interrupts_lib.o)
 .data          0x00000000        0x0 C:/Program Files/Microchip/mplabc32/v1.12/bin/../lib/gcc/pic32mx/3.4.4/../../../../pic32mx/lib\libmchp_peripheral_32MX360F512L.a(int_disable_interrupts_lib.o)
 .bss           0x00000000        0x0 C:/Program Files/Microchip/mplabc32/v1.12/bin/../lib/gcc/pic32mx/3.4.4/../../../../pic32mx/lib\libmchp_peripheral_32MX360F512L.a(int_disable_interrupts_lib.o)
 .reginfo       0x00000000       0x18 C:/Program Files/Microchip/mplabc32/v1.12/bin/../lib/gcc/pic32mx/3.4.4/../../../../pic32mx/lib\libmchp_peripheral_32MX360F512L.a(int_disable_interrupts_lib.o)
 .pdr           0x00000000       0x20 C:/Program Files/Microchip/mplabc32/v1.12/bin/../lib/gcc/pic32mx/3.4.4/../../../../pic32mx/lib\libmchp_peripheral_32MX360F512L.a(int_disable_interrupts_lib.o)
 .text          0x00000000        0x0 C:/Program Files/Microchip/mplabc32/v1.12/bin/../lib/gcc/pic32mx/3.4.4/../../../../pic32mx/lib\libmchp_peripheral_32MX360F512L.a(int_restore_interrupts_lib.o)
 .data          0x00000000        0x0 C:/Program Files/Microchip/mplabc32/v1.12/bin/../lib/gcc/pic32mx/3.4.4/../../../../pic32mx/lib\libmchp_peripheral_32MX360F512L.a(int_restore_interrupts_lib.o)
 .bss           0x00000000        0x0 C:/Program Files/Microchip/mplabc32/v1.12/bin/../lib/gcc/pic32mx/3.4.4/../../../../pic32mx/lib\libmchp_peripheral_32MX360F512L.a(int_restore_interrupts_lib.o)
 .reginfo       0x00000000       0x18 C:/Program Files/Microchip/mplabc32/v1.12/bin/../lib/gcc/pic32mx/3.4.4/../../../../pic32mx/lib\libmchp_peripheral_32MX360F512L.a(int_restore_interrupts_lib.o)
 .pdr           0x00000000       0x20 C:/Program Files/Microchip/mplabc32/v1.12/bin/../lib/gcc/pic32mx/3.4.4/../../../../pic32mx/lib\libmchp_peripheral_32MX360F512L.a(int_restore_interrupts_lib.o)
 .text          0x00000000        0x0 C:/Program Files/Microchip/mplabc32/v1.12/bin/../lib/gcc/pic32mx/3.4.4/../../../../pic32mx/lib\libmchp_peripheral_32MX360F512L.a(int_enable_mv_int_lib.o)
 .data          0x00000000        0x0 C:/Program Files/Microchip/mplabc32/v1.12/bin/../lib/gcc/pic32mx/3.4.4/../../../../pic32mx/lib\libmchp_peripheral_32MX360F512L.a(int_enable_mv_int_lib.o)
 .bss           0x00000000        0x0 C:/Program Files/Microchip/mplabc32/v1.12/bin/../lib/gcc/pic32mx/3.4.4/../../../../pic32mx/lib\libmchp_peripheral_32MX360F512L.a(int_enable_mv_int_lib.o)
 .reginfo       0x00000000       0x18 C:/Program Files/Microchip/mplabc32/v1.12/bin/../lib/gcc/pic32mx/3.4.4/../../../../pic32mx/lib\libmchp_peripheral_32MX360F512L.a(int_enable_mv_int_lib.o)
 .pdr           0x00000000       0x20 C:/Program Files/Microchip/mplabc32/v1.12/bin/../lib/gcc/pic32mx/3.4.4/../../../../pic32mx/lib\libmchp_peripheral_32MX360F512L.a(int_enable_mv_int_lib.o)
 .text          0x00000000        0x0 C:/Program Files/Microchip/mplabc32/v1.12/bin/../lib/gcc/pic32mx/3.4.4/../../../../pic32mx/lib\libmchp_peripheral_32MX360F512L.a(spi_getc_spi2_lib_legacy.o)
 .data          0x00000000        0x0 C:/Program Files/Microchip/mplabc32/v1.12/bin/../lib/gcc/pic32mx/3.4.4/../../../../pic32mx/lib\libmchp_peripheral_32MX360F512L.a(spi_getc_spi2_lib_legacy.o)
 .bss           0x00000000        0x0 C:/Program Files/Microchip/mplabc32/v1.12/bin/../lib/gcc/pic32mx/3.4.4/../../../../pic32mx/lib\libmchp_peripheral_32MX360F512L.a(spi_getc_spi2_lib_legacy.o)
 .reginfo       0x00000000       0x18 C:/Program Files/Microchip/mplabc32/v1.12/bin/../lib/gcc/pic32mx/3.4.4/../../../../pic32mx/lib\libmchp_peripheral_32MX360F512L.a(spi_getc_spi2_lib_legacy.o)
 .pdr           0x00000000       0x20 C:/Program Files/Microchip/mplabc32/v1.12/bin/../lib/gcc/pic32mx/3.4.4/../../../../pic32mx/lib\libmchp_peripheral_32MX360F512L.a(spi_getc_spi2_lib_legacy.o)
 .text          0x00000000        0x0 C:/Program Files/Microchip/mplabc32/v1.12/bin/../lib/gcc/pic32mx/3.4.4/../../../../pic32mx/lib\libmchp_peripheral_32MX360F512L.a(spi_open_spi2_lib_legacy.o)
 .data          0x00000000        0x0 C:/Program Files/Microchip/mplabc32/v1.12/bin/../lib/gcc/pic32mx/3.4.4/../../../../pic32mx/lib\libmchp_peripheral_32MX360F512L.a(spi_open_spi2_lib_legacy.o)
 .bss           0x00000000        0x0 C:/Program Files/Microchip/mplabc32/v1.12/bin/../lib/gcc/pic32mx/3.4.4/../../../../pic32mx/lib\libmchp_peripheral_32MX360F512L.a(spi_open_spi2_lib_legacy.o)
 .reginfo       0x00000000       0x18 C:/Program Files/Microchip/mplabc32/v1.12/bin/../lib/gcc/pic32mx/3.4.4/../../../../pic32mx/lib\libmchp_peripheral_32MX360F512L.a(spi_open_spi2_lib_legacy.o)
 .pdr           0x00000000       0x20 C:/Program Files/Microchip/mplabc32/v1.12/bin/../lib/gcc/pic32mx/3.4.4/../../../../pic32mx/lib\libmchp_peripheral_32MX360F512L.a(spi_open_spi2_lib_legacy.o)
 .text          0x00000000        0x0 C:/Program Files/Microchip/mplabc32/v1.12/bin/../lib/gcc/pic32mx/3.4.4/../../../../pic32mx/lib\libmchp_peripheral_32MX360F512L.a(spi_brg_tbl_lib_legacy.o)
 .data          0x00000000        0x0 C:/Program Files/Microchip/mplabc32/v1.12/bin/../lib/gcc/pic32mx/3.4.4/../../../../pic32mx/lib\libmchp_peripheral_32MX360F512L.a(spi_brg_tbl_lib_legacy.o)
 .bss           0x00000000        0x0 C:/Program Files/Microchip/mplabc32/v1.12/bin/../lib/gcc/pic32mx/3.4.4/../../../../pic32mx/lib\libmchp_peripheral_32MX360F512L.a(spi_brg_tbl_lib_legacy.o)
 .reginfo       0x00000000       0x18 C:/Program Files/Microchip/mplabc32/v1.12/bin/../lib/gcc/pic32mx/3.4.4/../../../../pic32mx/lib\libmchp_peripheral_32MX360F512L.a(spi_brg_tbl_lib_legacy.o)
 .pdr           0x00000000        0x0 C:/Program Files/Microchip/mplabc32/v1.12/bin/../lib/gcc/pic32mx/3.4.4/../../../../pic32mx/lib\libmchp_peripheral_32MX360F512L.a(spi_brg_tbl_lib_legacy.o)
 .text          0x00000000        0x0 C:/Program Files/Microchip/mplabc32/v1.12/bin/../lib/gcc/pic32mx/3.4.4/../../../../pic32mx/lib\libmchp_peripheral_32MX360F512L.a(int_enable_interrupts_lib.o)
 .data          0x00000000        0x0 C:/Program Files/Microchip/mplabc32/v1.12/bin/../lib/gcc/pic32mx/3.4.4/../../../../pic32mx/lib\libmchp_peripheral_32MX360F512L.a(int_enable_interrupts_lib.o)
 .bss           0x00000000        0x0 C:/Program Files/Microchip/mplabc32/v1.12/bin/../lib/gcc/pic32mx/3.4.4/../../../../pic32mx/lib\libmchp_peripheral_32MX360F512L.a(int_enable_interrupts_lib.o)
 .reginfo       0x00000000       0x18 C:/Program Files/Microchip/mplabc32/v1.12/bin/../lib/gcc/pic32mx/3.4.4/../../../../pic32mx/lib\libmchp_peripheral_32MX360F512L.a(int_enable_interrupts_lib.o)
 .pdr           0x00000000       0x20 C:/Program Files/Microchip/mplabc32/v1.12/bin/../lib/gcc/pic32mx/3.4.4/../../../../pic32mx/lib\libmchp_peripheral_32MX360F512L.a(int_enable_interrupts_lib.o)
 .text          0x00000000        0x0 C:/Program Files/Microchip/mplabc32/v1.12/bin/../lib/gcc/pic32mx/3.4.4/../../../../pic32mx/lib\libc.a(doprnt_cdnopsuxX.eo)
 .data          0x00000000        0x0 C:/Program Files/Microchip/mplabc32/v1.12/bin/../lib/gcc/pic32mx/3.4.4/../../../../pic32mx/lib\libc.a(doprnt_cdnopsuxX.eo)
 .bss           0x00000000        0x0 C:/Program Files/Microchip/mplabc32/v1.12/bin/../lib/gcc/pic32mx/3.4.4/../../../../pic32mx/lib\libc.a(doprnt_cdnopsuxX.eo)
 .reginfo       0x00000000       0x18 C:/Program Files/Microchip/mplabc32/v1.12/bin/../lib/gcc/pic32mx/3.4.4/../../../../pic32mx/lib\libc.a(doprnt_cdnopsuxX.eo)
 .pdr           0x00000000       0x20 C:/Program Files/Microchip/mplabc32/v1.12/bin/../lib/gcc/pic32mx/3.4.4/../../../../pic32mx/lib\libc.a(doprnt_cdnopsuxX.eo)
 .data          0x00000000        0x0 C:/Program Files/Microchip/mplabc32/v1.12/bin/../lib/gcc/pic32mx/3.4.4\libgcc.a(_udivdi3.o)
 .bss           0x00000000        0x0 C:/Program Files/Microchip/mplabc32/v1.12/bin/../lib/gcc/pic32mx/3.4.4\libgcc.a(_udivdi3.o)
 .reginfo       0x00000000       0x18 C:/Program Files/Microchip/mplabc32/v1.12/bin/../lib/gcc/pic32mx/3.4.4\libgcc.a(_udivdi3.o)
 .pdr           0x00000000       0x20 C:/Program Files/Microchip/mplabc32/v1.12/bin/../lib/gcc/pic32mx/3.4.4\libgcc.a(_udivdi3.o)
 .data          0x00000000        0x0 C:/Program Files/Microchip/mplabc32/v1.12/bin/../lib/gcc/pic32mx/3.4.4\libgcc.a(_umoddi3.o)
 .bss           0x00000000        0x0 C:/Program Files/Microchip/mplabc32/v1.12/bin/../lib/gcc/pic32mx/3.4.4\libgcc.a(_umoddi3.o)
 .reginfo       0x00000000       0x18 C:/Program Files/Microchip/mplabc32/v1.12/bin/../lib/gcc/pic32mx/3.4.4\libgcc.a(_umoddi3.o)
 .pdr           0x00000000       0x20 C:/Program Files/Microchip/mplabc32/v1.12/bin/../lib/gcc/pic32mx/3.4.4\libgcc.a(_umoddi3.o)
 .text          0x00000000        0x0 C:/Program Files/Microchip/mplabc32/v1.12/bin/../lib/gcc/pic32mx/3.4.4/../../../../pic32mx/lib/./proc/32MX360F512L\processor.o
 .data          0x00000000        0x0 C:/Program Files/Microchip/mplabc32/v1.12/bin/../lib/gcc/pic32mx/3.4.4/../../../../pic32mx/lib/./proc/32MX360F512L\processor.o
 .bss           0x00000000        0x0 C:/Program Files/Microchip/mplabc32/v1.12/bin/../lib/gcc/pic32mx/3.4.4/../../../../pic32mx/lib/./proc/32MX360F512L\processor.o
 .reginfo       0x00000000       0x18 C:/Program Files/Microchip/mplabc32/v1.12/bin/../lib/gcc/pic32mx/3.4.4/../../../../pic32mx/lib/./proc/32MX360F512L\processor.o
 .pdr           0x00000000        0x0 C:/Program Files/Microchip/mplabc32/v1.12/bin/../lib/gcc/pic32mx/3.4.4/../../../../pic32mx/lib/./proc/32MX360F512L\processor.o

Memory Configuration

Name             Origin             Length             Attributes
kseg0_program_mem 0x9d000000         0x00080000         xr
kseg0_boot_mem   0x9fc00490         0x00000970
exception_mem    0x9fc01000         0x00001000
kseg1_boot_mem   0xbfc00000         0x00000490
debug_exec_mem   0xbfc02000         0x00000ff0
config3          0xbfc02ff0         0x00000004
config2          0xbfc02ff4         0x00000004
config1          0xbfc02ff8         0x00000004
config0          0xbfc02ffc         0x00000004
kseg1_data_mem   0xa0000000         0x00008000         w !x
sfrs             0xbf800000         0x00100000
configsfrs       0xbfc02ff0         0x00000010
*default*        0x00000000         0xffffffff

Linker script and memory map

LOAD C:/Program Files/Microchip/mplabc32/v1.12/bin/../lib/gcc/pic32mx/3.4.4/../../../../pic32mx/lib/crt0.o
LOAD output_pic32_ssd1963\Application.o
LOAD output_pic32_ssd1963\Primitive.o
LOAD output_pic32_ssd1963\GOLFontDefault.o
LOAD output_pic32_ssd1963\JpegDecoder.o
LOAD output_pic32_ssd1963\BmpDecoder.o
LOAD output_pic32_ssd1963\GifDecoder.o
LOAD output_pic32_ssd1963\ImageDecoder.o
LOAD output_pic32_ssd1963\jidctint.o
LOAD output_pic32_ssd1963\DisplayDriver.o
LOAD output_pic32_ssd1963\SD-SPI.o
LOAD output_pic32_ssd1963\FSIO.o
LOAD output_pic32_ssd1963\GOLMediumlFont.o
LOAD output_pic32_ssd1963\GOLSmallFont.o
                0x00000001                __MPLAB_BUILD = 0x1
                0x00002000                _min_heap_size = 0x2000
                0x00000800                _min_stack_size = 0x800
LOAD C:/Program Files/Microchip/mplabc32/v1.12/bin/../lib/gcc/pic32mx/3.4.4\libgcc.a
START GROUP
LOAD C:/Program Files/Microchip/mplabc32/v1.12/bin/../lib/gcc/pic32mx/3.4.4/../../../../pic32mx/lib\libdebug.a
LOAD C:/Program Files/Microchip/mplabc32/v1.12/bin/../lib/gcc/pic32mx/3.4.4/../../../../pic32mx/lib\libc.a
LOAD C:/Program Files/Microchip/mplabc32/v1.12/bin/../lib/gcc/pic32mx/3.4.4/../../../../pic32mx/lib\libm.a
LOAD C:/Program Files/Microchip/mplabc32/v1.12/bin/../lib/gcc/pic32mx/3.4.4/../../../../pic32mx/lib\libe.a
LOAD C:/Program Files/Microchip/mplabc32/v1.12/bin/../lib/gcc/pic32mx/3.4.4/../../../../pic32mx/lib\libdsp.a
LOAD C:/Program Files/Microchip/mplabc32/v1.12/bin/../lib/gcc/pic32mx/3.4.4/../../../../pic32mx/lib\libmchp_peripheral.a
LOAD C:/Program Files/Microchip/mplabc32/v1.12/bin/../lib/gcc/pic32mx/3.4.4/../../../../pic32mx/lib\libmchp_peripheral_32MX360F512L.a
END GROUP
LOAD C:/Program Files/Microchip/mplabc32/v1.12/bin/../lib/gcc/pic32mx/3.4.4\libgcc.a
                0x00000400                PROVIDE (_min_stack_size, 0x400)
                0x00000000                PROVIDE (_min_heap_size, 0x0)
LOAD C:/Program Files/Microchip/mplabc32/v1.12/bin/../lib/gcc/pic32mx/3.4.4/../../../../pic32mx/lib/./proc/32MX360F512L\processor.o
                0x00000001                PROVIDE (_vector_spacing, 0x1)
                0x9fc01000                _ebase_address = 0x9fc01000
                0xbfc00000                _RESET_ADDR = 0xbfc00000
                0xbfc00380                _BEV_EXCPT_ADDR = 0xbfc00380
                0xbfc00480                _DBG_EXCPT_ADDR = 0xbfc00480
                0xbfc02000                _DBG_CODE_ADDR = 0xbfc02000
                0x9fc01180                _GEN_EXCPT_ADDR = (_ebase_address + 0x180)

.config_BFC02FF0
 *(.config_BFC02FF0)

.config_BFC02FF4
                0xbfc02ff4        0x4
 *(.config_BFC02FF4)
 .config_BFC02FF4
                0xbfc02ff4        0x4 output_pic32_ssd1963\Application.o

.config_BFC02FF8
                0xbfc02ff8        0x4
 *(.config_BFC02FF8)
 .config_BFC02FF8
                0xbfc02ff8        0x4 output_pic32_ssd1963\Application.o

.config_BFC02FFC
                0xbfc02ffc        0x4
 *(.config_BFC02FFC)
 .config_BFC02FFC
                0xbfc02ffc        0x4 output_pic32_ssd1963\Application.o

.reset          0xbfc00000       0x10
 *(.reset)
 .reset         0xbfc00000       0x10 C:/Program Files/Microchip/mplabc32/v1.12/bin/../lib/gcc/pic32mx/3.4.4/../../../../pic32mx/lib/crt0.o
                0xbfc00000                _reset

.bev_excpt      0xbfc00380       0x10
 *(.bev_handler)
 .bev_handler   0xbfc00380       0x10 C:/Program Files/Microchip/mplabc32/v1.12/bin/../lib/gcc/pic32mx/3.4.4/../../../../pic32mx/lib/crt0.o

.dbg_excpt      0xbfc00480        0x0
                0xbfc00480                . = (. + DEFINED (_DEBUGGER)?0x8:0x0)

.dbg_code       0xbfc02000        0x0
                0xbfc02000                . = (. + DEFINED (_DEBUGGER)?0xff0:0x0)

.app_excpt      0x9fc01180       0x10
 *(.gen_handler)
 .gen_handler   0x9fc01180       0x10 C:/Program Files/Microchip/mplabc32/v1.12/bin/../lib/gcc/pic32mx/3.4.4/../../../../pic32mx/lib/crt0.o

.vector_0       0x9fc01200        0x0
 *(.vector_0)
                0x00000001                ASSERT (((_vector_spacing == 0x0) || (SIZEOF (.vector_0) <= (_vector_spacing << 0x5))), function at exception vector 0 too large)

.vector_1       0x9fc01220        0x0
 *(.vector_1)
                0x00000001                ASSERT (((_vector_spacing == 0x0) || (SIZEOF (.vector_1) <= (_vector_spacing << 0x5))), function at exception vector 1 too large)

.vector_2       0x9fc01240        0x0
 *(.vector_2)
                0x00000001                ASSERT (((_vector_spacing == 0x0) || (SIZEOF (.vector_2) <= (_vector_spacing << 0x5))), function at exception vector 2 too large)

.vector_3       0x9fc01260        0x0
 *(.vector_3)
                0x00000001                ASSERT (((_vector_spacing == 0x0) || (SIZEOF (.vector_3) <= (_vector_spacing << 0x5))), function at exception vector 3 too large)

.vector_4       0x9fc01280        0x0
 *(.vector_4)
                0x00000001                ASSERT (((_vector_spacing == 0x0) || (SIZEOF (.vector_4) <= (_vector_spacing << 0x5))), function at exception vector 4 too large)

.vector_5       0x9fc012a0        0x0
 *(.vector_5)
                0x00000001                ASSERT (((_vector_spacing == 0x0) || (SIZEOF (.vector_5) <= (_vector_spacing << 0x5))), function at exception vector 5 too large)

.vector_6       0x9fc012c0        0x0
 *(.vector_6)
                0x00000001                ASSERT (((_vector_spacing == 0x0) || (SIZEOF (.vector_6) <= (_vector_spacing << 0x5))), function at exception vector 6 too large)

.vector_7       0x9fc012e0        0x0
 *(.vector_7)
                0x00000001                ASSERT (((_vector_spacing == 0x0) || (SIZEOF (.vector_7) <= (_vector_spacing << 0x5))), function at exception vector 7 too large)

.vector_8       0x9fc01300        0x0
 *(.vector_8)
                0x00000001                ASSERT (((_vector_spacing == 0x0) || (SIZEOF (.vector_8) <= (_vector_spacing << 0x5))), function at exception vector 8 too large)

.vector_9       0x9fc01320        0x0
 *(.vector_9)
                0x00000001                ASSERT (((_vector_spacing == 0x0) || (SIZEOF (.vector_9) <= (_vector_spacing << 0x5))), function at exception vector 9 too large)

.vector_10      0x9fc01340        0x0
 *(.vector_10)
                0x00000001                ASSERT (((_vector_spacing == 0x0) || (SIZEOF (.vector_10) <= (_vector_spacing << 0x5))), function at exception vector 10 too large)

.vector_11      0x9fc01360        0x0
 *(.vector_11)
                0x00000001                ASSERT (((_vector_spacing == 0x0) || (SIZEOF (.vector_11) <= (_vector_spacing << 0x5))), function at exception vector 11 too large)

.vector_12      0x9fc01380        0x0
 *(.vector_12)
                0x00000001                ASSERT (((_vector_spacing == 0x0) || (SIZEOF (.vector_12) <= (_vector_spacing << 0x5))), function at exception vector 12 too large)

.vector_13      0x9fc013a0        0x0
 *(.vector_13)
                0x00000001                ASSERT (((_vector_spacing == 0x0) || (SIZEOF (.vector_13) <= (_vector_spacing << 0x5))), function at exception vector 13 too large)

.vector_14      0x9fc013c0        0x0
 *(.vector_14)
                0x00000001                ASSERT (((_vector_spacing == 0x0) || (SIZEOF (.vector_14) <= (_vector_spacing << 0x5))), function at exception vector 14 too large)

.vector_15      0x9fc013e0        0x0
 *(.vector_15)
                0x00000001                ASSERT (((_vector_spacing == 0x0) || (SIZEOF (.vector_15) <= (_vector_spacing << 0x5))), function at exception vector 15 too large)

.vector_16      0x9fc01400        0x0
 *(.vector_16)
                0x00000001                ASSERT (((_vector_spacing == 0x0) || (SIZEOF (.vector_16) <= (_vector_spacing << 0x5))), function at exception vector 16 too large)

.vector_17      0x9fc01420        0x0
 *(.vector_17)
                0x00000001                ASSERT (((_vector_spacing == 0x0) || (SIZEOF (.vector_17) <= (_vector_spacing << 0x5))), function at exception vector 17 too large)

.vector_18      0x9fc01440        0x0
 *(.vector_18)
                0x00000001                ASSERT (((_vector_spacing == 0x0) || (SIZEOF (.vector_18) <= (_vector_spacing << 0x5))), function at exception vector 18 too large)

.vector_19      0x9fc01460        0x0
 *(.vector_19)
                0x00000001                ASSERT (((_vector_spacing == 0x0) || (SIZEOF (.vector_19) <= (_vector_spacing << 0x5))), function at exception vector 19 too large)

.vector_20      0x9fc01480        0x0
 *(.vector_20)
                0x00000001                ASSERT (((_vector_spacing == 0x0) || (SIZEOF (.vector_20) <= (_vector_spacing << 0x5))), function at exception vector 20 too large)

.vector_21      0x9fc014a0        0x0
 *(.vector_21)
                0x00000001                ASSERT (((_vector_spacing == 0x0) || (SIZEOF (.vector_21) <= (_vector_spacing << 0x5))), function at exception vector 21 too large)

.vector_22      0x9fc014c0        0x0
 *(.vector_22)
                0x00000001                ASSERT (((_vector_spacing == 0x0) || (SIZEOF (.vector_22) <= (_vector_spacing << 0x5))), function at exception vector 22 too large)

.vector_23      0x9fc014e0        0x0
 *(.vector_23)
                0x00000001                ASSERT (((_vector_spacing == 0x0) || (SIZEOF (.vector_23) <= (_vector_spacing << 0x5))), function at exception vector 23 too large)

.vector_24      0x9fc01500        0x0
 *(.vector_24)
                0x00000001                ASSERT (((_vector_spacing == 0x0) || (SIZEOF (.vector_24) <= (_vector_spacing << 0x5))), function at exception vector 24 too large)

.vector_25      0x9fc01520        0x0
 *(.vector_25)
                0x00000001                ASSERT (((_vector_spacing == 0x0) || (SIZEOF (.vector_25) <= (_vector_spacing << 0x5))), function at exception vector 25 too large)

.vector_26      0x9fc01540        0x0
 *(.vector_26)
                0x00000001                ASSERT (((_vector_spacing == 0x0) || (SIZEOF (.vector_26) <= (_vector_spacing << 0x5))), function at exception vector 26 too large)

.vector_27      0x9fc01560        0x0
 *(.vector_27)
                0x00000001                ASSERT (((_vector_spacing == 0x0) || (SIZEOF (.vector_27) <= (_vector_spacing << 0x5))), function at exception vector 27 too large)

.vector_28      0x9fc01580        0x0
 *(.vector_28)
                0x00000001                ASSERT (((_vector_spacing == 0x0) || (SIZEOF (.vector_28) <= (_vector_spacing << 0x5))), function at exception vector 28 too large)

.vector_29      0x9fc015a0        0x0
 *(.vector_29)
                0x00000001                ASSERT (((_vector_spacing == 0x0) || (SIZEOF (.vector_29) <= (_vector_spacing << 0x5))), function at exception vector 29 too large)

.vector_30      0x9fc015c0        0x0
 *(.vector_30)
                0x00000001                ASSERT (((_vector_spacing == 0x0) || (SIZEOF (.vector_30) <= (_vector_spacing << 0x5))), function at exception vector 30 too large)

.vector_31      0x9fc015e0        0x0
 *(.vector_31)
                0x00000001                ASSERT (((_vector_spacing == 0x0) || (SIZEOF (.vector_31) <= (_vector_spacing << 0x5))), function at exception vector 31 too large)

.vector_32      0x9fc01600        0x0
 *(.vector_32)
                0x00000001                ASSERT (((_vector_spacing == 0x0) || (SIZEOF (.vector_32) <= (_vector_spacing << 0x5))), function at exception vector 32 too large)

.vector_33      0x9fc01620        0x0
 *(.vector_33)
                0x00000001                ASSERT (((_vector_spacing == 0x0) || (SIZEOF (.vector_33) <= (_vector_spacing << 0x5))), function at exception vector 33 too large)

.vector_34      0x9fc01640        0x0
 *(.vector_34)
                0x00000001                ASSERT (((_vector_spacing == 0x0) || (SIZEOF (.vector_34) <= (_vector_spacing << 0x5))), function at exception vector 34 too large)

.vector_35      0x9fc01660        0x0
 *(.vector_35)
                0x00000001                ASSERT (((_vector_spacing == 0x0) || (SIZEOF (.vector_35) <= (_vector_spacing << 0x5))), function at exception vector 35 too large)

.vector_36      0x9fc01680        0x0
 *(.vector_36)
                0x00000001                ASSERT (((_vector_spacing == 0x0) || (SIZEOF (.vector_36) <= (_vector_spacing << 0x5))), function at exception vector 36 too large)

.vector_37      0x9fc016a0        0x0
 *(.vector_37)
                0x00000001                ASSERT (((_vector_spacing == 0x0) || (SIZEOF (.vector_37) <= (_vector_spacing << 0x5))), function at exception vector 37 too large)

.vector_38      0x9fc016c0        0x0
 *(.vector_38)
                0x00000001                ASSERT (((_vector_spacing == 0x0) || (SIZEOF (.vector_38) <= (_vector_spacing << 0x5))), function at exception vector 38 too large)

.vector_39      0x9fc016e0        0x0
 *(.vector_39)
                0x00000001                ASSERT (((_vector_spacing == 0x0) || (SIZEOF (.vector_39) <= (_vector_spacing << 0x5))), function at exception vector 39 too large)

.vector_40      0x9fc01700        0x0
 *(.vector_40)
                0x00000001                ASSERT (((_vector_spacing == 0x0) || (SIZEOF (.vector_40) <= (_vector_spacing << 0x5))), function at exception vector 40 too large)

.vector_41      0x9fc01720        0x0
 *(.vector_41)
                0x00000001                ASSERT (((_vector_spacing == 0x0) || (SIZEOF (.vector_41) <= (_vector_spacing << 0x5))), function at exception vector 41 too large)

.vector_42      0x9fc01740        0x0
 *(.vector_42)
                0x00000001                ASSERT (((_vector_spacing == 0x0) || (SIZEOF (.vector_42) <= (_vector_spacing << 0x5))), function at exception vector 42 too large)

.vector_43      0x9fc01760        0x0
 *(.vector_43)
                0x00000001                ASSERT (((_vector_spacing == 0x0) || (SIZEOF (.vector_43) <= (_vector_spacing << 0x5))), function at exception vector 43 too large)

.vector_44      0x9fc01780        0x0
 *(.vector_44)
                0x00000001                ASSERT (((_vector_spacing == 0x0) || (SIZEOF (.vector_44) <= (_vector_spacing << 0x5))), function at exception vector 44 too large)

.vector_45      0x9fc017a0        0x0
 *(.vector_45)
                0x00000001                ASSERT (((_vector_spacing == 0x0) || (SIZEOF (.vector_45) <= (_vector_spacing << 0x5))), function at exception vector 45 too large)

.vector_46      0x9fc017c0        0x0
 *(.vector_46)
                0x00000001                ASSERT (((_vector_spacing == 0x0) || (SIZEOF (.vector_46) <= (_vector_spacing << 0x5))), function at exception vector 46 too large)

.vector_47      0x9fc017e0        0x0
 *(.vector_47)
                0x00000001                ASSERT (((_vector_spacing == 0x0) || (SIZEOF (.vector_47) <= (_vector_spacing << 0x5))), function at exception vector 47 too large)

.vector_48      0x9fc01800        0x0
 *(.vector_48)
                0x00000001                ASSERT (((_vector_spacing == 0x0) || (SIZEOF (.vector_48) <= (_vector_spacing << 0x5))), function at exception vector 48 too large)

.vector_49      0x9fc01820        0x0
 *(.vector_49)
                0x00000001                ASSERT (((_vector_spacing == 0x0) || (SIZEOF (.vector_49) <= (_vector_spacing << 0x5))), function at exception vector 49 too large)

.vector_50      0x9fc01840        0x0
 *(.vector_50)
                0x00000001                ASSERT (((_vector_spacing == 0x0) || (SIZEOF (.vector_50) <= (_vector_spacing << 0x5))), function at exception vector 50 too large)

.vector_51      0x9fc01860        0x0
 *(.vector_51)
                0x00000001                ASSERT (((_vector_spacing == 0x0) || (SIZEOF (.vector_51) <= (_vector_spacing << 0x5))), function at exception vector 51 too large)

.vector_52      0x9fc01880        0x0
 *(.vector_52)
                0x00000001                ASSERT (((_vector_spacing == 0x0) || (SIZEOF (.vector_52) <= (_vector_spacing << 0x5))), function at exception vector 52 too large)

.vector_53      0x9fc018a0        0x0
 *(.vector_53)
                0x00000001                ASSERT (((_vector_spacing == 0x0) || (SIZEOF (.vector_53) <= (_vector_spacing << 0x5))), function at exception vector 53 too large)

.vector_54      0x9fc018c0        0x0
 *(.vector_54)
                0x00000001                ASSERT (((_vector_spacing == 0x0) || (SIZEOF (.vector_54) <= (_vector_spacing << 0x5))), function at exception vector 54 too large)

.vector_55      0x9fc018e0        0x0
 *(.vector_55)
                0x00000001                ASSERT (((_vector_spacing == 0x0) || (SIZEOF (.vector_55) <= (_vector_spacing << 0x5))), function at exception vector 55 too large)

.vector_56      0x9fc01900        0x0
 *(.vector_56)
                0x00000001                ASSERT (((_vector_spacing == 0x0) || (SIZEOF (.vector_56) <= (_vector_spacing << 0x5))), function at exception vector 56 too large)

.vector_57      0x9fc01920        0x0
 *(.vector_57)
                0x00000001                ASSERT (((_vector_spacing == 0x0) || (SIZEOF (.vector_57) <= (_vector_spacing << 0x5))), function at exception vector 57 too large)

.vector_58      0x9fc01940        0x0
 *(.vector_58)
                0x00000001                ASSERT (((_vector_spacing == 0x0) || (SIZEOF (.vector_58) <= (_vector_spacing << 0x5))), function at exception vector 58 too large)

.vector_59      0x9fc01960        0x0
 *(.vector_59)
                0x00000001                ASSERT (((_vector_spacing == 0x0) || (SIZEOF (.vector_59) <= (_vector_spacing << 0x5))), function at exception vector 59 too large)

.vector_60      0x9fc01980        0x0
 *(.vector_60)
                0x00000001                ASSERT (((_vector_spacing == 0x0) || (SIZEOF (.vector_60) <= (_vector_spacing << 0x5))), function at exception vector 60 too large)

.vector_61      0x9fc019a0        0x0
 *(.vector_61)
                0x00000001                ASSERT (((_vector_spacing == 0x0) || (SIZEOF (.vector_61) <= (_vector_spacing << 0x5))), function at exception vector 61 too large)

.vector_62      0x9fc019c0        0x0
 *(.vector_62)
                0x00000001                ASSERT (((_vector_spacing == 0x0) || (SIZEOF (.vector_62) <= (_vector_spacing << 0x5))), function at exception vector 62 too large)

.vector_63      0x9fc019e0        0x0
 *(.vector_63)
                0x00000001                ASSERT (((_vector_spacing == 0x0) || (SIZEOF (.vector_63) <= (_vector_spacing << 0x5))), function at exception vector 63 too large)

.startup        0x9fc00490      0x1e0
 *(.startup)
 .startup       0x9fc00490      0x1e0 C:/Program Files/Microchip/mplabc32/v1.12/bin/../lib/gcc/pic32mx/3.4.4/../../../../pic32mx/lib/crt0.o

.text           0x9d000000    0x11d20
                0x9d000000                _text_begin = .
 *(.text .stub .text.* .gnu.linkonce.t.*)
 .text          0x9d000000       0x10 C:/Program Files/Microchip/mplabc32/v1.12/bin/../lib/gcc/pic32mx/3.4.4/../../../../pic32mx/lib/crt0.o
                0x9d000008                __crt0_exit
 .text          0x9d000010      0xad8 output_pic32_ssd1963\Application.o
                0x9d000010                PixelOutput
                0x9d0000ac                main
 .text          0x9d000ae8     0x1528 output_pic32_ssd1963\Primitive.o
                0x9d000ae8                InitGraph
                0x9d000b58                Arc
                0x9d0011b8                Line
                0x9d001538                Bevel
                0x9d001968                FillBevel
                0x9d001b9c                DrawPoly
                0x9d001c54                SetFont
                0x9d001c88                OutText
                0x9d001ce8                OutTextXY
                0x9d001d10                OutChar
                0x9d001f20                GetTextWidth
                0x9d001fb0                GetTextHeight
                0x9d001fd0                GetImageWidth
                0x9d001ff0                GetImageHeight
 .text          0x9d002010     0x1ba0 output_pic32_ssd1963\JpegDecoder.o
                0x9d003a30                JPEG_bDecode
 .text          0x9d003bb0     0x15c4 output_pic32_ssd1963\BmpDecoder.o
                0x9d003bb0                BDEC_vResetData
                0x9d003be8                BDEC_bReadHeader
                0x9d003f10                BMP_bDecode
 .text          0x9d005174      0xfdc output_pic32_ssd1963\GifDecoder.o
                0x9d0060e4                GIF_bDecode
 .text          0x9d006150      0x208 output_pic32_ssd1963\ImageDecoder.o
                0x9d006150                ImageDecoderInit
                0x9d006174                ImageLoopCallbackRegister
                0x9d00617c                ImageDecode
                0x9d006230                IMG_vSetboundaries
 .text          0x9d006358      0x520 output_pic32_ssd1963\jidctint.o
                0x9d006358                jpeg_idct_islow
 .text          0x9d006878     0x237c output_pic32_ssd1963\DisplayDriver.o
                0x9d006878                DelayMs
                0x9d006b08                SetArea
                0x9d006d58                SetScrollArea
                0x9d006edc                SetScrollStart
                0x9d006fb0                EnterSleepMode
                0x9d007014                ExitSleepMode
                0x9d007078                DisplayOff
                0x9d0070dc                DisplayOn
                0x9d007140                EnterDeepSleep
                0x9d0071a4                SetBacklight
                0x9d00731c                SetTearingCfg
                0x9d007434                ResetDevice
                0x9d007f14                PutPixel
                0x9d008020                GetPixel
                0x9d008028                Bar
                0x9d0081c0                ClearDevice
                0x9d0082c4                PutImage
                0x9d008380                PutImage1BPP
                0x9d0085a0                PutImage4BPP
                0x9d0087ec                PutImage8BPP
                0x9d008a10                PutImage16BPP
 .text          0x9d008bf4      0xaa8 output_pic32_ssd1963\SD-SPI.o
                0x9d008bf4                MDD_SDSPI_MediaDetect
                0x9d008c08                MDD_SDSPI_ReadSectorSize
                0x9d008c10                MDD_SDSPI_ReadCapacity
                0x9d008c18                MDD_SDSPI_InitIO
                0x9d008c60                MDD_SDSPI_ShutdownMedia
                0x9d008c90                SendMMCCmd
                0x9d008f20                MDD_SDSPI_SectorRead
                0x9d009084                MDD_SDSPI_SectorWrite
                0x9d0091d4                MDD_SDSPI_WriteProtectState
                0x9d0091e4                Delayms
                0x9d009228                CloseSPIM
                0x9d009240                WriteSPIM
                0x9d00927c                MDD_SDSPI_ReadMedia
                0x9d0092b8                OpenSPIM
                0x9d009324                MDD_SDSPI_MediaInitialize
 .text          0x9d00969c     0x674c output_pic32_ssd1963\FSIO.o
                0x9d00969c                FSInit
                0x9d009788                FILEfind
                0x9d009a2c                FILEopen
                0x9d009bc0                FILEget_next_cluster
                0x9d009c94                DISKmount
                0x9d009d48                LoadMBR
                0x9d009f9c                LoadBootSector
                0x9d00a294                GetFullClusterNumber
                0x9d00a2a8                FSCreateMBR
                0x9d00a4d4                FSformat
                0x9d00ae14                Write_File_Entry
                0x9d00aed8                FAT_erase_cluster_chain
                0x9d00b018                Cache_File_Entry
                0x9d00b290                CreateFileEntry
                0x9d00b340                CreateFirstCluster
                0x9d00b3bc                FindEmptyEntries
                0x9d00b52c                PopulateEntries
                0x9d00b664                CacheTime
                0x9d00b798                FILEallocate_new_cluster
                0x9d00b880                FATfindEmptyCluster
                0x9d00b994                FSfclose
                0x9d00bae8                Fill_File_Object
                0x9d00bc58                LoadDirAttrib
                0x9d00bd14                FILEerase
                0x9d00be24                FSrename
                0x9d00c078                FSfopen
                0x9d00c50c                FSftell
                0x9d00c518                FSremove
                0x9d00c638                FSrewind
                0x9d00c680                FSerror
                0x9d00c688                FileObjectCopy
                0x9d00c6bc                FILECreateHeadCluster
                0x9d00c7b4                EraseCluster
                0x9d00c8b0                ReadByte
                0x9d00c8c0                ReadWord
                0x9d00c8dc                ReadDWord
                0x9d00c934                Cluster2Sector
                0x9d00c9ac                FSattrib
                0x9d00ca7c                FSfwrite
                0x9d00cda4                flushData
                0x9d00ce08                FSfeof
                0x9d00ce20                FSfread
                0x9d00d034                FormatFileName
                0x9d00d1b4                FormatDirName
                0x9d00d350                ValidateChars
                0x9d00d4e8                FSfseek
                0x9d00d704                ReadFAT
                0x9d00d9ec                WriteFAT
                0x9d00dd44                FSchdir
                0x9d00dd68                chdirhelper
                0x9d00e22c                FSgetcwd
                0x9d00e688                GetPreviousEntry
                0x9d00e890                FSmkdir
                0x9d00e8b4                mkdirhelper
                0x9d00ed54                CreateDIR
                0x9d00eed8                writeDotEntries
                0x9d00f068                FSrmdir
                0x9d00f094                rmdirhelper
                0x9d00f81c                eraseDir
                0x9d00f8f8                FindFirst
                0x9d00fb9c                FindNext
 .text          0x9d00fde8       0xa8 C:/Program Files/Microchip/mplabc32/v1.12/bin/../lib/gcc/pic32mx/3.4.4/../../../../pic32mx/lib\libc.a(memset.o)
                0x9d00fde8                memset
 .text          0x9d00fe90      0x1a0 C:/Program Files/Microchip/mplabc32/v1.12/bin/../lib/gcc/pic32mx/3.4.4/../../../../pic32mx/lib\libc.a(strcpy.o)
                0x9d00fe90                strcpy
 .text          0x9d010030      0x168 C:/Program Files/Microchip/mplabc32/v1.12/bin/../lib/gcc/pic32mx/3.4.4/../../../../pic32mx/lib\libc.a(strlen.o)
                0x9d010030                strlen
 .text.general_exception
                0x9d010198       0xd0 C:/Program Files/Microchip/mplabc32/v1.12/bin/../lib/gcc/pic32mx/3.4.4/../../../../pic32mx/lib\libc.a(general-exception.o)
                0x9d010198                _general_exception_context
 .text.tolower  0x9d010268       0x20 C:/Program Files/Microchip/mplabc32/v1.12/bin/../lib/gcc/pic32mx/3.4.4/../../../../pic32mx/lib\libc.a(ctypef.o)
                0x9d010268                tolower
 .text.toupper  0x9d010288       0x20 C:/Program Files/Microchip/mplabc32/v1.12/bin/../lib/gcc/pic32mx/3.4.4/../../../../pic32mx/lib\libc.a(ctypef.o)
                0x9d010288                toupper
 .text.fputs    0x9d0102a8       0x7c C:/Program Files/Microchip/mplabc32/v1.12/bin/../lib/gcc/pic32mx/3.4.4/../../../../pic32mx/lib\libc.a(puts.o)
                0x9d0102a8                fputs
 .text.puts     0x9d010324       0x48 C:/Program Files/Microchip/mplabc32/v1.12/bin/../lib/gcc/pic32mx/3.4.4/../../../../pic32mx/lib\libc.a(puts.o)
                0x9d010324                puts
 .text.strchr   0x9d01036c       0x28 C:/Program Files/Microchip/mplabc32/v1.12/bin/../lib/gcc/pic32mx/3.4.4/../../../../pic32mx/lib\libc.a(strchr.o)
                0x9d01036c                strchr
 .text.strncpy  0x9d010394       0x48 C:/Program Files/Microchip/mplabc32/v1.12/bin/../lib/gcc/pic32mx/3.4.4/../../../../pic32mx/lib\libc.a(strncpy.o)
                0x9d010394                strncpy
 .text._printf_cdnopuxX
                0x9d0103dc       0x38 C:/Program Files/Microchip/mplabc32/v1.12/bin/../lib/gcc/pic32mx/3.4.4/../../../../pic32mx/lib\libc.a(printf_cdnopuxX.eo)
                0x9d0103dc                _printf_cdnopuxX
 .text._sprintf_s
                0x9d010414       0x60 C:/Program Files/Microchip/mplabc32/v1.12/bin/../lib/gcc/pic32mx/3.4.4/../../../../pic32mx/lib\libc.a(sprintf_s.eo)
                0x9d010414                _sprintf_0
                0x9d010414                _sprintf_s
 .text._general_exception_handler
                0x9d010474        0x8 C:/Program Files/Microchip/mplabc32/v1.12/bin/../lib/gcc/pic32mx/3.4.4/../../../../pic32mx/lib\libc.a(default-general-exception-handler.o)
                0x9d010474                _general_exception_handler
 .text._bootstrap_exception_handler
                0x9d01047c        0x8 C:/Program Files/Microchip/mplabc32/v1.12/bin/../lib/gcc/pic32mx/3.4.4/../../../../pic32mx/lib\libc.a(default-bootstrap-exception-handler.o)
                0x9d01047c                _bootstrap_exception_handler
 .text._on_reset
                0x9d010484        0x8 C:/Program Files/Microchip/mplabc32/v1.12/bin/../lib/gcc/pic32mx/3.4.4/../../../../pic32mx/lib\libc.a(default-on-reset.o)
                0x9d010484                _on_reset
 .text._on_bootstrap
                0x9d01048c        0x8 C:/Program Files/Microchip/mplabc32/v1.12/bin/../lib/gcc/pic32mx/3.4.4/../../../../pic32mx/lib\libc.a(default-on-bootstrap.o)
                0x9d01048c                _on_bootstrap
 .text          0x9d010494       0x18 C:/Program Files/Microchip/mplabc32/v1.12/bin/../lib/gcc/pic32mx/3.4.4/../../../../pic32mx/lib\libc.a(default-nmi-handler.o)
                0x9d010494                _nmi_handler
 .text.fputc    0x9d0104ac      0x144 C:/Program Files/Microchip/mplabc32/v1.12/bin/../lib/gcc/pic32mx/3.4.4/../../../../pic32mx/lib\libc.a(_fputc_simple.o)
                0x9d0104ac                fputc
 .text.write    0x9d0105f0       0xa8 C:/Program Files/Microchip/mplabc32/v1.12/bin/../lib/gcc/pic32mx/3.4.4/../../../../pic32mx/lib\libc.a(write.o)
                0x9d0105f0                write
 .text._flsbuf  0x9d010698      0x12c C:/Program Files/Microchip/mplabc32/v1.12/bin/../lib/gcc/pic32mx/3.4.4/../../../../pic32mx/lib\libc.a(_flsbuf_simple.o)
                0x9d010698                _flsbuf
 .text._mon_putc
                0x9d0107c4       0xa4 C:/Program Files/Microchip/mplabc32/v1.12/bin/../lib/gcc/pic32mx/3.4.4/../../../../pic32mx/lib\libc.a(_mon_putc.o)
                0x9d0107c4                _mon_putc
 .text.OpenCoreTimer
                0x9d010868        0xc C:/Program Files/Microchip/mplabc32/v1.12/bin/../lib/gcc/pic32mx/3.4.4/../../../../pic32mx/lib\libmchp_peripheral.a(open_core_timer_lib.o)
                0x9d010868                OpenCoreTimer
 .text.CheKseg0CacheOn
                0x9d010874       0x18 C:/Program Files/Microchip/mplabc32/v1.12/bin/../lib/gcc/pic32mx/3.4.4/../../../../pic32mx/lib\libmchp_peripheral_32MX360F512L.a(pcache.o)
                0x9d010874                CheKseg0CacheOn
 .text.INTDisableInterrupts
                0x9d01088c        0x8 C:/Program Files/Microchip/mplabc32/v1.12/bin/../lib/gcc/pic32mx/3.4.4/../../../../pic32mx/lib\libmchp_peripheral_32MX360F512L.a(int_disable_interrupts_lib.o)
                0x9d01088c                INTDisableInterrupts
 .text.INTRestoreInterrupts
                0x9d010894       0x1c C:/Program Files/Microchip/mplabc32/v1.12/bin/../lib/gcc/pic32mx/3.4.4/../../../../pic32mx/lib\libmchp_peripheral_32MX360F512L.a(int_restore_interrupts_lib.o)
                0x9d010894                INTRestoreInterrupts
 .text.INTEnableSystemMultiVectoredInt
                0x9d0108b0       0x34 C:/Program Files/Microchip/mplabc32/v1.12/bin/../lib/gcc/pic32mx/3.4.4/../../../../pic32mx/lib\libmchp_peripheral_32MX360F512L.a(int_enable_mv_int_lib.o)
                0x9d0108b0                INTEnableSystemMultiVectoredInt
 .text.getcSPI2
                0x9d0108e4       0x24 C:/Program Files/Microchip/mplabc32/v1.12/bin/../lib/gcc/pic32mx/3.4.4/../../../../pic32mx/lib\libmchp_peripheral_32MX360F512L.a(spi_getc_spi2_lib_legacy.o)
                0x9d0108e4                getcSPI2
 .text.OpenSPI2
                0x9d010908       0x64 C:/Program Files/Microchip/mplabc32/v1.12/bin/../lib/gcc/pic32mx/3.4.4/../../../../pic32mx/lib\libmchp_peripheral_32MX360F512L.a(spi_open_spi2_lib_legacy.o)
                0x9d010908                OpenSPI2
 .text.INTEnableInterrupts
                0x9d01096c        0x8 C:/Program Files/Microchip/mplabc32/v1.12/bin/../lib/gcc/pic32mx/3.4.4/../../../../pic32mx/lib\libmchp_peripheral_32MX360F512L.a(int_enable_interrupts_lib.o)
                0x9d01096c                INTEnableInterrupts
 .text._vfprintf_cdnopsuxX
                0x9d010974      0xaa4 C:/Program Files/Microchip/mplabc32/v1.12/bin/../lib/gcc/pic32mx/3.4.4/../../../../pic32mx/lib\libc.a(doprnt_cdnopsuxX.eo)
                0x9d010974                _vfprintf_0
                0x9d010974                _vfprintf_cdnopuxX
                0x9d010974                _vfprintf_cdnopsuxX
                0x9d010974                _vfprintf_s
 .text          0x9d011418      0x47c C:/Program Files/Microchip/mplabc32/v1.12/bin/../lib/gcc/pic32mx/3.4.4\libgcc.a(_udivdi3.o)
                0x9d011418                __udivdi3
 .text          0x9d011894      0x48c C:/Program Files/Microchip/mplabc32/v1.12/bin/../lib/gcc/pic32mx/3.4.4\libgcc.a(_umoddi3.o)
                0x9d011894                __umoddi3
 *(.text.*personality*)
 *(.gnu.warning)
 *(.mips16.fn.*)
 *(.mips16.call.*)
                0x9d011d20                _text_end = .

.rodata         0x9d011d20     0x25a4
 *(.rodata .rodata.* .gnu.linkonce.r.*)
 .rodata.str1.4
                0x9d011d20      0x1f9 output_pic32_ssd1963\Application.o
                                0x1fc (size before relaxing)
 *fill*         0x9d011f19        0x3 00
 .rodata        0x9d011f1c     0x1588 output_pic32_ssd1963\GOLFontDefault.o
                0x9d011f1c                GOLFontDefault
                0x9d011f24                L11903
 .rodata        0x9d0134a4       0x50 output_pic32_ssd1963\JpegDecoder.o
 .rodata        0x9d0134f4       0x1c output_pic32_ssd1963\GifDecoder.o
 .rodata        0x9d013510       0xd8 output_pic32_ssd1963\SD-SPI.o
                0x9d013510                sdmmc_cmdtable
 .rodata        0x9d0135e8       0xec output_pic32_ssd1963\FSIO.o
 .rodata.str1.4
                0x9d0136d4        0x3 output_pic32_ssd1963\FSIO.o
                                  0x4 (size before relaxing)
 *fill*         0x9d0136d7        0x1 00
 .rodata        0x9d0136d8      0x860 output_pic32_ssd1963\GOLSmallFont.o
                0x9d0136d8                GOLSmallFont
                0x9d0136e0                L25988
 .rodata        0x9d013f38      0x104 C:/Program Files/Microchip/mplabc32/v1.12/bin/../lib/gcc/pic32mx/3.4.4/../../../../pic32mx/lib\libc.a(ctype.o)
                0x9d013f38                _ctype
 .rodata._SpiBrgConvTbl
                0x9d01403c       0x80 C:/Program Files/Microchip/mplabc32/v1.12/bin/../lib/gcc/pic32mx/3.4.4/../../../../pic32mx/lib\libmchp_peripheral_32MX360F512L.a(spi_brg_tbl_lib_legacy.o)
                0x9d01403c                _SpiBrgConvTbl
 *fill*         0x9d0140bc        0x4 00
 .rodata        0x9d0140c0      0x1d0 C:/Program Files/Microchip/mplabc32/v1.12/bin/../lib/gcc/pic32mx/3.4.4/../../../../pic32mx/lib\libc.a(doprnt_cdnopsuxX.eo)
 .rodata.str1.4
                0x9d014290       0x30 C:/Program Files/Microchip/mplabc32/v1.12/bin/../lib/gcc/pic32mx/3.4.4/../../../../pic32mx/lib\libc.a(doprnt_cdnopsuxX.eo)
 .rodata.cst4   0x9d0142c0        0x4 C:/Program Files/Microchip/mplabc32/v1.12/bin/../lib/gcc/pic32mx/3.4.4/../../../../pic32mx/lib\libc.a(doprnt_cdnopsuxX.eo)
 *(.rodata1)
                0x9d0142c4                . = ALIGN (0x4)

.sdata2         0x9d0142c4        0x0
 *(.sdata2 .sdata2.* .gnu.linkonce.s2.*)
                0x9d0142c4                . = ALIGN (0x4)

.sbss2          0x9d0142c4        0x0
 *(.sbss2 .sbss2.* .gnu.linkonce.sb2.*)
                0x9d0142c4                . = ALIGN (0x4)

.eh_frame_hdr
 *(.eh_frame_hdr)

.eh_frame       0x9d0142c4       0x40
 *(.eh_frame)
 .eh_frame      0x9d0142c4       0x20 C:/Program Files/Microchip/mplabc32/v1.12/bin/../lib/gcc/pic32mx/3.4.4\libgcc.a(_udivdi3.o)
 .eh_frame      0x9d0142e4       0x20 C:/Program Files/Microchip/mplabc32/v1.12/bin/../lib/gcc/pic32mx/3.4.4\libgcc.a(_umoddi3.o)

.dbg_data       0xa0000000        0x0
                0xa0000000                . = (. + DEFINED (_DEBUGGER)?0x200:0x0)

.persist        0xa0000000        0x0
                0xa0000000                _persist_begin = .
 *(.persist .persist.*)
                0xa0000000                _persist_end = .

.data           0xa0000000       0xa0 load address 0x9d014304
                0xa0000000                _data_begin = .
 *(.data .data.* .gnu.linkonce.d.*)
 .data          0xa0000000       0xa0 C:/Program Files/Microchip/mplabc32/v1.12/bin/../lib/gcc/pic32mx/3.4.4/../../../../pic32mx/lib\libc.a(_iob.o)
                0xa0000000                _iob
 *(.gnu.linkonce.d.*personality*)
 *(.data1)
                0x9d014304                _data_image_begin = LOADADDR (.data)

.eh_frame
 *(.eh_frame)
                0xa00000a0                . = .
                0xa0008090                _gp = (ALIGN (0x10) + 0x7ff0)

.got
 *(.got.plt)
 *(.got)

.sdata          0xa00000a0       0x14 load address 0x9d0143a4
                0xa00000a0                _sdata_begin = .
 *(.sdata .sdata.* .gnu.linkonce.s.*)
 .sdata         0xa00000a0        0x1 output_pic32_ssd1963\Application.o
                0xa00000a0                panelBrightness
 *fill*         0xa00000a1        0x3 00
 .sdata         0xa00000a4        0xc output_pic32_ssd1963\FSIO.o
                0xa00000a4                gLastFATSectorRead
                0xa00000a8                gLastDataSectorRead
                0xa00000ac                cwdptr
 .sdata         0xa00000b0        0x4 C:/Program Files/Microchip/mplabc32/v1.12/bin/../lib/gcc/pic32mx/3.4.4/../../../../pic32mx/lib\libc.a(c32_uart.o)
                0xa00000b0                __C32_UART
                0xa00000b4                _sdata_end = .

.lit8
 *(.lit8)

.lit4
 *(.lit4)
                0xa00000b4                . = ALIGN (0x4)
                0xa00000b4                _data_end = .
                0xa00000b4                _bss_begin = .

.sbss           0xa00000b4       0x79 load address 0x9d0143b8
                0xa00000b4                _sbss_begin = .
 *(.dynsbss)
 *(.sbss .sbss.* .gnu.linkonce.sb.*)
 .sbss          0xa00000b4        0x1 output_pic32_ssd1963\DisplayDriver.o
                0xa00000b4                _gpioStatus
 *fill*         0xa00000b5        0x3 00
 .sbss          0xa00000b8        0x8 output_pic32_ssd1963\SD-SPI.o
 .sbss          0xa00000c0        0xc output_pic32_ssd1963\FSIO.o
                0xa00000c0                gNeedFATWrite
                0xa00000c4                gBufferOwner
                0xa00000c8                gNeedDataWrite
                0xa00000c9                nextClusterIsLast
                0xa00000ca                gBufferZeroed
                0xa00000cb                recache
 *(.scommon)
 .scommon       0xa00000cc       0x13 output_pic32_ssd1963\Primitive.o
                0xa00000cc                _cursorY
                0xa00000ce                _fontOrientation
                0xa00000d0                _fontFirstChar
                0xa00000d2                _fontHeight
                0xa00000d4                _cursorX
                0xa00000d6                _fontLastChar
                0xa00000d8                _font
                0xa00000dc                _lineType
                0xa00000de                _lineThickness
 *fill*         0xa00000df        0x1 00
 .scommon       0xa00000e0       0x18 output_pic32_ssd1963\ImageDecoder.o
                0xa00000e0                IMG_wWidth
                0xa00000e2                IMG_bAlignCenter
                0xa00000e4                IMG_wStartX
                0xa00000e6                IMG_wHeight
                0xa00000e8                IMG_bDownScalingFactor
                0xa00000ea                IMG_wStartY
                0xa00000ec                IMG_wImageWidth
                0xa00000ee                IMG_wImageHeight
                0xa00000f0                IMG_blAbortImageDecoding
                0xa00000f4                IMG_pLoopCallbackFn
 .scommon       0xa00000f8       0x10 output_pic32_ssd1963\DisplayDriver.o
                0xa00000f8                _activePage
                0xa00000fa                _clipRgn
                0xa00000fc                _visualPage
                0xa00000fe                _clipRight
                0xa0000100                _clipBottom
                0xa0000102                _clipTop
                0xa0000104                _color
                0xa0000106                _clipLeft
 .scommon       0xa0000108        0x7 output_pic32_ssd1963\SD-SPI.o
                0xa0000108                MDD_SDSPI_finalLBA
                0xa000010c                gMediaSectorSize
                0xa000010e                gSDMode
 *fill*         0xa000010f        0x1 00
 .scommon       0xa0000110       0x1c output_pic32_ssd1963\FSIO.o
                0xa0000110                gFileSlotOpen
                0xa0000113                gTimeCrtMS
                0xa0000114                gTimeCrtTime
                0xa0000118                FatRootDirClusterValue
                0xa000011c                gTimeWrtDate
                0xa000011e                gTimeCrtDate
                0xa0000120                TempClusterCalc
                0xa0000124                dirCleared
                0xa0000126                gTimeAccDate
                0xa0000128                FSerrno
                0xa000012a                gTimeWrtTime
 .scommon       0xa000012c        0x1 C:/Program Files/Microchip/mplabc32/v1.12/bin/../lib/gcc/pic32mx/3.4.4/../../../../pic32mx/lib\libc.a(_iob.o)
                0xa000012c                _outdone
                0xa000012d                _sbss_end = .

.bss            0xa0000130      0x5ec load address 0x9d0143b8
 *(.dynbss)
 *(.bss .bss.* .gnu.linkonce.b.*)
 *(COMMON)
 COMMON         0xa0000130      0x5aa output_pic32_ssd1963\FSIO.o
                0xa0000130                gDataBuffer
                0xa0000330                cwd
                0xa000036c                defaultString
                0xa000037c                tempCWDobj
                0xa00003b8                gFATBuffer
                0xa00005b8                gFileArray
                0xa000066c                gDiskData
                0xa0000694                gFileTemp
                0xa00006d0                defaultArray
 *fill*         0xa00006da        0x2 00
 COMMON         0xa00006dc       0x40 C:/Program Files/Microchip/mplabc32/v1.12/bin/../lib/gcc/pic32mx/3.4.4/../../../../pic32mx/lib\libc.a(_iob.o)
                0xa00006dc                _sibuf
                0xa00006fc                _sobuf
                0xa000071c                . = ALIGN (0x4)
                0xa000071c                . = ALIGN (0x4)
                0xa000071c                _end = .
                0xa000071c                _bss_end = .

.heap           0xa0000720     0x2000 load address 0x9d0143b8
                0xa0000720                _heap = .
                0xa0002720                . = (. + _min_heap_size)
 *fill*         0xa0000720     0x2000 00
                0xa0002720                . = ALIGN (0x8)

.stack          0xa0002720      0x800 load address 0x9d0143b8
                0xa0002720                _splim = .
                0xa0002720                _SPLIM = .
                0xa0002f20                . = (. + _min_stack_size)
 *fill*         0xa0002720      0x800 00
                0xa0002f20                . = ALIGN (0x8)

.ramfunc        0xa0003000        0x0 load address 0x9d0143b8
                0xa0003000                _ramfunc_begin = .
 *(.ramfunc .ramfunc.*)
                0xa0003000                . = ALIGN (0x4)
                0xa0003000                _ramfunc_end = .
                0x9d0143b8                _ramfunc_image_begin = LOADADDR (.ramfunc)
                0x00000000                _ramfunc_length = SIZEOF (.ramfunc)
                0x00003000                _bmxdkpba_address = (_ramfunc_begin - 0xa0000000)
                0x00008000                _bmxdudba_address = 0x8000
                0x00008000                _bmxdupba_address = 0x8000
                0xa0008000                _stack = (_ramfunc_length > 0x0)?(_ramfunc_begin - 0x8):0xa0008000
                0x00000001                ASSERT (((_min_stack_size + _min_heap_size) <= (_stack - _heap)), Not enough space to allocate both stack and heap.  Reduce heap and/or stack size.)

/DISCARD/
 *(.pdr)
 *(.reginfo)
 *(.rel.dyn)
 *(.note.GNU-stack)

.stab
 *(.stab)

.stabstr
 *(.stabstr)

.stab.excl
 *(.stab.excl)

.stab.exclstr
 *(.stab.exclstr)

.stab.index
 *(.stab.index)

.stab.indexstr
 *(.stab.indexstr)

.mdebug.abi32   0x00000000        0x0
 .mdebug.abi32  0x00000000        0x0 output_pic32_ssd1963\Application.o
 .mdebug.abi32  0x00000000        0x0 output_pic32_ssd1963\Primitive.o
 .mdebug.abi32  0x00000000        0x0 output_pic32_ssd1963\GOLFontDefault.o
 .mdebug.abi32  0x00000000        0x0 output_pic32_ssd1963\JpegDecoder.o
 .mdebug.abi32  0x00000000        0x0 output_pic32_ssd1963\BmpDecoder.o
 .mdebug.abi32  0x00000000        0x0 output_pic32_ssd1963\GifDecoder.o
 .mdebug.abi32  0x00000000        0x0 output_pic32_ssd1963\ImageDecoder.o
 .mdebug.abi32  0x00000000        0x0 output_pic32_ssd1963\jidctint.o
 .mdebug.abi32  0x00000000        0x0 output_pic32_ssd1963\DisplayDriver.o
 .mdebug.abi32  0x00000000        0x0 output_pic32_ssd1963\SD-SPI.o
 .mdebug.abi32  0x00000000        0x0 output_pic32_ssd1963\FSIO.o
 .mdebug.abi32  0x00000000        0x0 output_pic32_ssd1963\GOLMediumlFont.o
 .mdebug.abi32  0x00000000        0x0 output_pic32_ssd1963\GOLSmallFont.o
 .mdebug.abi32  0x00000000        0x0 C:/Program Files/Microchip/mplabc32/v1.12/bin/../lib/gcc/pic32mx/3.4.4/../../../../pic32mx/lib\libc.a(ctypef.o)
 .mdebug.abi32  0x00000000        0x0 C:/Program Files/Microchip/mplabc32/v1.12/bin/../lib/gcc/pic32mx/3.4.4/../../../../pic32mx/lib\libc.a(puts.o)
 .mdebug.abi32  0x00000000        0x0 C:/Program Files/Microchip/mplabc32/v1.12/bin/../lib/gcc/pic32mx/3.4.4/../../../../pic32mx/lib\libc.a(strchr.o)
 .mdebug.abi32  0x00000000        0x0 C:/Program Files/Microchip/mplabc32/v1.12/bin/../lib/gcc/pic32mx/3.4.4/../../../../pic32mx/lib\libc.a(strncpy.o)
 .mdebug.abi32  0x00000000        0x0 C:/Program Files/Microchip/mplabc32/v1.12/bin/../lib/gcc/pic32mx/3.4.4/../../../../pic32mx/lib\libc.a(printf_cdnopuxX.eo)
 .mdebug.abi32  0x00000000        0x0 C:/Program Files/Microchip/mplabc32/v1.12/bin/../lib/gcc/pic32mx/3.4.4/../../../../pic32mx/lib\libc.a(sprintf_s.eo)
 .mdebug.abi32  0x00000000        0x0 C:/Program Files/Microchip/mplabc32/v1.12/bin/../lib/gcc/pic32mx/3.4.4/../../../../pic32mx/lib\libc.a(default-general-exception-handler.o)
 .mdebug.abi32  0x00000000        0x0 C:/Program Files/Microchip/mplabc32/v1.12/bin/../lib/gcc/pic32mx/3.4.4/../../../../pic32mx/lib\libc.a(default-bootstrap-exception-handler.o)
 .mdebug.abi32  0x00000000        0x0 C:/Program Files/Microchip/mplabc32/v1.12/bin/../lib/gcc/pic32mx/3.4.4/../../../../pic32mx/lib\libc.a(default-on-reset.o)
 .mdebug.abi32  0x00000000        0x0 C:/Program Files/Microchip/mplabc32/v1.12/bin/../lib/gcc/pic32mx/3.4.4/../../../../pic32mx/lib\libc.a(default-on-bootstrap.o)
 .mdebug.abi32  0x00000000        0x0 C:/Program Files/Microchip/mplabc32/v1.12/bin/../lib/gcc/pic32mx/3.4.4/../../../../pic32mx/lib\libc.a(_iob.o)
 .mdebug.abi32  0x00000000        0x0 C:/Program Files/Microchip/mplabc32/v1.12/bin/../lib/gcc/pic32mx/3.4.4/../../../../pic32mx/lib\libc.a(_fputc_simple.o)
 .mdebug.abi32  0x00000000        0x0 C:/Program Files/Microchip/mplabc32/v1.12/bin/../lib/gcc/pic32mx/3.4.4/../../../../pic32mx/lib\libc.a(ctype.o)
 .mdebug.abi32  0x00000000        0x0 C:/Program Files/Microchip/mplabc32/v1.12/bin/../lib/gcc/pic32mx/3.4.4/../../../../pic32mx/lib\libc.a(write.o)
 .mdebug.abi32  0x00000000        0x0 C:/Program Files/Microchip/mplabc32/v1.12/bin/../lib/gcc/pic32mx/3.4.4/../../../../pic32mx/lib\libc.a(_flsbuf_simple.o)
 .mdebug.abi32  0x00000000        0x0 C:/Program Files/Microchip/mplabc32/v1.12/bin/../lib/gcc/pic32mx/3.4.4/../../../../pic32mx/lib\libc.a(_mon_putc.o)
 .mdebug.abi32  0x00000000        0x0 C:/Program Files/Microchip/mplabc32/v1.12/bin/../lib/gcc/pic32mx/3.4.4/../../../../pic32mx/lib\libc.a(c32_uart.o)
 .mdebug.abi32  0x00000000        0x0 C:/Program Files/Microchip/mplabc32/v1.12/bin/../lib/gcc/pic32mx/3.4.4/../../../../pic32mx/lib\libmchp_peripheral.a(open_core_timer_lib.o)
 .mdebug.abi32  0x00000000        0x0 C:/Program Files/Microchip/mplabc32/v1.12/bin/../lib/gcc/pic32mx/3.4.4/../../../../pic32mx/lib\libmchp_peripheral_32MX360F512L.a(pcache.o)
 .mdebug.abi32  0x00000000        0x0 C:/Program Files/Microchip/mplabc32/v1.12/bin/../lib/gcc/pic32mx/3.4.4/../../../../pic32mx/lib\libmchp_peripheral_32MX360F512L.a(int_disable_interrupts_lib.o)
 .mdebug.abi32  0x00000000        0x0 C:/Program Files/Microchip/mplabc32/v1.12/bin/../lib/gcc/pic32mx/3.4.4/../../../../pic32mx/lib\libmchp_peripheral_32MX360F512L.a(int_restore_interrupts_lib.o)
 .mdebug.abi32  0x00000000        0x0 C:/Program Files/Microchip/mplabc32/v1.12/bin/../lib/gcc/pic32mx/3.4.4/../../../../pic32mx/lib\libmchp_peripheral_32MX360F512L.a(int_enable_mv_int_lib.o)
 .mdebug.abi32  0x00000000        0x0 C:/Program Files/Microchip/mplabc32/v1.12/bin/../lib/gcc/pic32mx/3.4.4/../../../../pic32mx/lib\libmchp_peripheral_32MX360F512L.a(spi_getc_spi2_lib_legacy.o)
 .mdebug.abi32  0x00000000        0x0 C:/Program Files/Microchip/mplabc32/v1.12/bin/../lib/gcc/pic32mx/3.4.4/../../../../pic32mx/lib\libmchp_peripheral_32MX360F512L.a(spi_open_spi2_lib_legacy.o)
 .mdebug.abi32  0x00000000        0x0 C:/Program Files/Microchip/mplabc32/v1.12/bin/../lib/gcc/pic32mx/3.4.4/../../../../pic32mx/lib\libmchp_peripheral_32MX360F512L.a(spi_brg_tbl_lib_legacy.o)
 .mdebug.abi32  0x00000000        0x0 C:/Program Files/Microchip/mplabc32/v1.12/bin/../lib/gcc/pic32mx/3.4.4/../../../../pic32mx/lib\libmchp_peripheral_32MX360F512L.a(int_enable_interrupts_lib.o)
 .mdebug.abi32  0x00000000        0x0 C:/Program Files/Microchip/mplabc32/v1.12/bin/../lib/gcc/pic32mx/3.4.4/../../../../pic32mx/lib\libc.a(doprnt_cdnopsuxX.eo)
 .mdebug.abi32  0x00000000        0x0 C:/Program Files/Microchip/mplabc32/v1.12/bin/../lib/gcc/pic32mx/3.4.4\libgcc.a(_udivdi3.o)
 .mdebug.abi32  0x00000000        0x0 C:/Program Files/Microchip/mplabc32/v1.12/bin/../lib/gcc/pic32mx/3.4.4\libgcc.a(_umoddi3.o)

.comment        0x00000000      0xe41
 *(.comment)
 .comment       0x00000000       0x4d output_pic32_ssd1963\Application.o
 .comment       0x0000004d       0x4d output_pic32_ssd1963\Primitive.o
 .comment       0x0000009a       0x4d output_pic32_ssd1963\GOLFontDefault.o
 .comment       0x000000e7       0x4d output_pic32_ssd1963\JpegDecoder.o
 .comment       0x00000134       0x4d output_pic32_ssd1963\BmpDecoder.o
 .comment       0x00000181       0x4d output_pic32_ssd1963\GifDecoder.o
 .comment       0x000001ce       0x4d output_pic32_ssd1963\ImageDecoder.o
 .comment       0x0000021b       0x4d output_pic32_ssd1963\jidctint.o
 .comment       0x00000268       0x4d output_pic32_ssd1963\DisplayDriver.o
 .comment       0x000002b5       0x4d output_pic32_ssd1963\SD-SPI.o
 .comment       0x00000302       0x4d output_pic32_ssd1963\FSIO.o
 .comment       0x0000034f       0x4d output_pic32_ssd1963\GOLMediumlFont.o
 .comment       0x0000039c       0x4d output_pic32_ssd1963\GOLSmallFont.o
 .comment       0x000003e9       0x56 C:/Program Files/Microchip/mplabc32/v1.12/bin/../lib/gcc/pic32mx/3.4.4/../../../../pic32mx/lib\libc.a(memset.o)
 .comment       0x0000043f       0x56 C:/Program Files/Microchip/mplabc32/v1.12/bin/../lib/gcc/pic32mx/3.4.4/../../../../pic32mx/lib\libc.a(strcpy.o)
 .comment       0x00000495       0x56 C:/Program Files/Microchip/mplabc32/v1.12/bin/../lib/gcc/pic32mx/3.4.4/../../../../pic32mx/lib\libc.a(strlen.o)
 .comment       0x000004eb       0x9c C:/Program Files/Microchip/mplabc32/v1.12/bin/../lib/gcc/pic32mx/3.4.4/../../../../pic32mx/lib\libc.a(ctypef.o)
 .comment       0x00000587       0x4d C:/Program Files/Microchip/mplabc32/v1.12/bin/../lib/gcc/pic32mx/3.4.4/../../../../pic32mx/lib\libc.a(puts.o)
 .comment       0x000005d4       0x4d C:/Program Files/Microchip/mplabc32/v1.12/bin/../lib/gcc/pic32mx/3.4.4/../../../../pic32mx/lib\libc.a(strchr.o)
 .comment       0x00000621       0x4d C:/Program Files/Microchip/mplabc32/v1.12/bin/../lib/gcc/pic32mx/3.4.4/../../../../pic32mx/lib\libc.a(strncpy.o)
 .comment       0x0000066e       0x4d C:/Program Files/Microchip/mplabc32/v1.12/bin/../lib/gcc/pic32mx/3.4.4/../../../../pic32mx/lib\libc.a(printf_cdnopuxX.eo)
 .comment       0x000006bb       0x4d C:/Program Files/Microchip/mplabc32/v1.12/bin/../lib/gcc/pic32mx/3.4.4/../../../../pic32mx/lib\libc.a(sprintf_s.eo)
 .comment       0x00000708       0x4d C:/Program Files/Microchip/mplabc32/v1.12/bin/../lib/gcc/pic32mx/3.4.4/../../../../pic32mx/lib\libc.a(default-general-exception-handler.o)
 .comment       0x00000755       0x4d C:/Program Files/Microchip/mplabc32/v1.12/bin/../lib/gcc/pic32mx/3.4.4/../../../../pic32mx/lib\libc.a(default-bootstrap-exception-handler.o)
 .comment       0x000007a2       0x4d C:/Program Files/Microchip/mplabc32/v1.12/bin/../lib/gcc/pic32mx/3.4.4/../../../../pic32mx/lib\libc.a(default-on-reset.o)
 .comment       0x000007ef       0x4d C:/Program Files/Microchip/mplabc32/v1.12/bin/../lib/gcc/pic32mx/3.4.4/../../../../pic32mx/lib\libc.a(default-on-bootstrap.o)
 .comment       0x0000083c       0x4d C:/Program Files/Microchip/mplabc32/v1.12/bin/../lib/gcc/pic32mx/3.4.4/../../../../pic32mx/lib\libc.a(_iob.o)
 .comment       0x00000889       0x4d C:/Program Files/Microchip/mplabc32/v1.12/bin/../lib/gcc/pic32mx/3.4.4/../../../../pic32mx/lib\libc.a(_fputc_simple.o)
 .comment       0x000008d6       0x9b C:/Program Files/Microchip/mplabc32/v1.12/bin/../lib/gcc/pic32mx/3.4.4/../../../../pic32mx/lib\libc.a(ctype.o)
 .comment       0x00000971       0x4d C:/Program Files/Microchip/mplabc32/v1.12/bin/../lib/gcc/pic32mx/3.4.4/../../../../pic32mx/lib\libc.a(write.o)
 .comment       0x000009be       0x4d C:/Program Files/Microchip/mplabc32/v1.12/bin/../lib/gcc/pic32mx/3.4.4/../../../../pic32mx/lib\libc.a(_flsbuf_simple.o)
 .comment       0x00000a0b       0x4d C:/Program Files/Microchip/mplabc32/v1.12/bin/../lib/gcc/pic32mx/3.4.4/../../../../pic32mx/lib\libc.a(_mon_putc.o)
 .comment       0x00000a58       0x4d C:/Program Files/Microchip/mplabc32/v1.12/bin/../lib/gcc/pic32mx/3.4.4/../../../../pic32mx/lib\libc.a(c32_uart.o)
 .comment       0x00000aa5       0x4d C:/Program Files/Microchip/mplabc32/v1.12/bin/../lib/gcc/pic32mx/3.4.4/../../../../pic32mx/lib\libmchp_peripheral.a(open_core_timer_lib.o)
 .comment       0x00000af2       0x4d C:/Program Files/Microchip/mplabc32/v1.12/bin/../lib/gcc/pic32mx/3.4.4/../../../../pic32mx/lib\libmchp_peripheral_32MX360F512L.a(pcache.o)
 .comment       0x00000b3f       0x4d C:/Program Files/Microchip/mplabc32/v1.12/bin/../lib/gcc/pic32mx/3.4.4/../../../../pic32mx/lib\libmchp_peripheral_32MX360F512L.a(int_disable_interrupts_lib.o)
 .comment       0x00000b8c       0x4d C:/Program Files/Microchip/mplabc32/v1.12/bin/../lib/gcc/pic32mx/3.4.4/../../../../pic32mx/lib\libmchp_peripheral_32MX360F512L.a(int_restore_interrupts_lib.o)
 .comment       0x00000bd9       0x4d C:/Program Files/Microchip/mplabc32/v1.12/bin/../lib/gcc/pic32mx/3.4.4/../../../../pic32mx/lib\libmchp_peripheral_32MX360F512L.a(int_enable_mv_int_lib.o)
 .comment       0x00000c26       0x4d C:/Program Files/Microchip/mplabc32/v1.12/bin/../lib/gcc/pic32mx/3.4.4/../../../../pic32mx/lib\libmchp_peripheral_32MX360F512L.a(spi_getc_spi2_lib_legacy.o)
 .comment       0x00000c73       0x4d C:/Program Files/Microchip/mplabc32/v1.12/bin/../lib/gcc/pic32mx/3.4.4/../../../../pic32mx/lib\libmchp_peripheral_32MX360F512L.a(spi_open_spi2_lib_legacy.o)
 .comment       0x00000cc0       0x4d C:/Program Files/Microchip/mplabc32/v1.12/bin/../lib/gcc/pic32mx/3.4.4/../../../../pic32mx/lib\libmchp_peripheral_32MX360F512L.a(spi_brg_tbl_lib_legacy.o)
 .comment       0x00000d0d       0x4d C:/Program Files/Microchip/mplabc32/v1.12/bin/../lib/gcc/pic32mx/3.4.4/../../../../pic32mx/lib\libmchp_peripheral_32MX360F512L.a(int_enable_interrupts_lib.o)
 .comment       0x00000d5a       0x4d C:/Program Files/Microchip/mplabc32/v1.12/bin/../lib/gcc/pic32mx/3.4.4/../../../../pic32mx/lib\libc.a(doprnt_cdnopsuxX.eo)
 .comment       0x00000da7       0x4d C:/Program Files/Microchip/mplabc32/v1.12/bin/../lib/gcc/pic32mx/3.4.4\libgcc.a(_udivdi3.o)
 .comment       0x00000df4       0x4d C:/Program Files/Microchip/mplabc32/v1.12/bin/../lib/gcc/pic32mx/3.4.4\libgcc.a(_umoddi3.o)

.debug
 *(.debug)

.line
 *(.line)

.debug_srcinfo
 *(.debug_srcinfo)

.debug_sfnames
 *(.debug_sfnames)

.debug_aranges  0x00000000      0x568
 *(.debug_aranges)
 .debug_aranges
                0x00000000       0x20 output_pic32_ssd1963\Application.o
 .debug_aranges
                0x00000020       0x20 output_pic32_ssd1963\Primitive.o
 .debug_aranges
                0x00000040       0x20 output_pic32_ssd1963\JpegDecoder.o
 .debug_aranges
                0x00000060       0x20 output_pic32_ssd1963\BmpDecoder.o
 .debug_aranges
                0x00000080       0x20 output_pic32_ssd1963\GifDecoder.o
 .debug_aranges
                0x000000a0       0x20 output_pic32_ssd1963\ImageDecoder.o
 .debug_aranges
                0x000000c0       0x20 output_pic32_ssd1963\jidctint.o
 .debug_aranges
                0x000000e0       0x20 output_pic32_ssd1963\DisplayDriver.o
 .debug_aranges
                0x00000100       0x20 output_pic32_ssd1963\SD-SPI.o
 .debug_aranges
                0x00000120       0x20 output_pic32_ssd1963\FSIO.o
 .debug_aranges
                0x00000140       0xa8 C:/Program Files/Microchip/mplabc32/v1.12/bin/../lib/gcc/pic32mx/3.4.4/../../../../pic32mx/lib\libc.a(ctypef.o)
 .debug_aranges
                0x000001e8       0x30 C:/Program Files/Microchip/mplabc32/v1.12/bin/../lib/gcc/pic32mx/3.4.4/../../../../pic32mx/lib\libc.a(puts.o)
 .debug_aranges
                0x00000218       0x28 C:/Program Files/Microchip/mplabc32/v1.12/bin/../lib/gcc/pic32mx/3.4.4/../../../../pic32mx/lib\libc.a(strchr.o)
 .debug_aranges
                0x00000240       0x28 C:/Program Files/Microchip/mplabc32/v1.12/bin/../lib/gcc/pic32mx/3.4.4/../../../../pic32mx/lib\libc.a(strncpy.o)
 .debug_aranges
                0x00000268       0x28 C:/Program Files/Microchip/mplabc32/v1.12/bin/../lib/gcc/pic32mx/3.4.4/../../../../pic32mx/lib\libc.a(printf_cdnopuxX.eo)
 .debug_aranges
                0x00000290       0x28 C:/Program Files/Microchip/mplabc32/v1.12/bin/../lib/gcc/pic32mx/3.4.4/../../../../pic32mx/lib\libc.a(sprintf_s.eo)
 .debug_aranges
                0x000002b8       0x28 C:/Program Files/Microchip/mplabc32/v1.12/bin/../lib/gcc/pic32mx/3.4.4/../../../../pic32mx/lib\libc.a(default-general-exception-handler.o)
 .debug_aranges
                0x000002e0       0x28 C:/Program Files/Microchip/mplabc32/v1.12/bin/../lib/gcc/pic32mx/3.4.4/../../../../pic32mx/lib\libc.a(default-bootstrap-exception-handler.o)
 .debug_aranges
                0x00000308       0x28 C:/Program Files/Microchip/mplabc32/v1.12/bin/../lib/gcc/pic32mx/3.4.4/../../../../pic32mx/lib\libc.a(default-on-reset.o)
 .debug_aranges
                0x00000330       0x28 C:/Program Files/Microchip/mplabc32/v1.12/bin/../lib/gcc/pic32mx/3.4.4/../../../../pic32mx/lib\libc.a(default-on-bootstrap.o)
 .debug_aranges
                0x00000358       0x28 C:/Program Files/Microchip/mplabc32/v1.12/bin/../lib/gcc/pic32mx/3.4.4/../../../../pic32mx/lib\libc.a(_fputc_simple.o)
 .debug_aranges
                0x00000380       0x28 C:/Program Files/Microchip/mplabc32/v1.12/bin/../lib/gcc/pic32mx/3.4.4/../../../../pic32mx/lib\libc.a(write.o)
 .debug_aranges
                0x000003a8       0x28 C:/Program Files/Microchip/mplabc32/v1.12/bin/../lib/gcc/pic32mx/3.4.4/../../../../pic32mx/lib\libc.a(_flsbuf_simple.o)
 .debug_aranges
                0x000003d0       0x28 C:/Program Files/Microchip/mplabc32/v1.12/bin/../lib/gcc/pic32mx/3.4.4/../../../../pic32mx/lib\libc.a(_mon_putc.o)
 .debug_aranges
                0x000003f8       0x28 C:/Program Files/Microchip/mplabc32/v1.12/bin/../lib/gcc/pic32mx/3.4.4/../../../../pic32mx/lib\libmchp_peripheral.a(open_core_timer_lib.o)
 .debug_aranges
                0x00000420       0x30 C:/Program Files/Microchip/mplabc32/v1.12/bin/../lib/gcc/pic32mx/3.4.4/../../../../pic32mx/lib\libmchp_peripheral_32MX360F512L.a(pcache.o)
 .debug_aranges
                0x00000450       0x28 C:/Program Files/Microchip/mplabc32/v1.12/bin/../lib/gcc/pic32mx/3.4.4/../../../../pic32mx/lib\libmchp_peripheral_32MX360F512L.a(int_disable_interrupts_lib.o)
 .debug_aranges
                0x00000478       0x28 C:/Program Files/Microchip/mplabc32/v1.12/bin/../lib/gcc/pic32mx/3.4.4/../../../../pic32mx/lib\libmchp_peripheral_32MX360F512L.a(int_restore_interrupts_lib.o)
 .debug_aranges
                0x000004a0       0x28 C:/Program Files/Microchip/mplabc32/v1.12/bin/../lib/gcc/pic32mx/3.4.4/../../../../pic32mx/lib\libmchp_peripheral_32MX360F512L.a(int_enable_mv_int_lib.o)
 .debug_aranges
                0x000004c8       0x28 C:/Program Files/Microchip/mplabc32/v1.12/bin/../lib/gcc/pic32mx/3.4.4/../../../../pic32mx/lib\libmchp_peripheral_32MX360F512L.a(spi_getc_spi2_lib_legacy.o)
 .debug_aranges
                0x000004f0       0x28 C:/Program Files/Microchip/mplabc32/v1.12/bin/../lib/gcc/pic32mx/3.4.4/../../../../pic32mx/lib\libmchp_peripheral_32MX360F512L.a(spi_open_spi2_lib_legacy.o)
 .debug_aranges
                0x00000518       0x28 C:/Program Files/Microchip/mplabc32/v1.12/bin/../lib/gcc/pic32mx/3.4.4/../../../../pic32mx/lib\libmchp_peripheral_32MX360F512L.a(int_enable_interrupts_lib.o)
 .debug_aranges
                0x00000540       0x28 C:/Program Files/Microchip/mplabc32/v1.12/bin/../lib/gcc/pic32mx/3.4.4/../../../../pic32mx/lib\libc.a(doprnt_cdnopsuxX.eo)

.debug_pubnames
                0x00000000     0x1227
 *(.debug_pubnames)
 .debug_pubnames
                0x00000000       0x3f output_pic32_ssd1963\Application.o
 .debug_pubnames
                0x0000003f      0x15f output_pic32_ssd1963\Primitive.o
 .debug_pubnames
                0x0000019e       0x30 output_pic32_ssd1963\GOLFontDefault.o
 .debug_pubnames
                0x000001ce       0x23 output_pic32_ssd1963\JpegDecoder.o
 .debug_pubnames
                0x000001f1       0x4b output_pic32_ssd1963\BmpDecoder.o
 .debug_pubnames
                0x0000023c       0x22 output_pic32_ssd1963\GifDecoder.o
 .debug_pubnames
                0x0000025e      0x139 output_pic32_ssd1963\ImageDecoder.o
 .debug_pubnames
                0x00000397       0x26 output_pic32_ssd1963\jidctint.o
 .debug_pubnames
                0x000003bd      0x1dd output_pic32_ssd1963\DisplayDriver.o
 .debug_pubnames
                0x0000059a      0x1ad output_pic32_ssd1963\SD-SPI.o
 .debug_pubnames
                0x00000747      0x5d9 output_pic32_ssd1963\FSIO.o
 .debug_pubnames
                0x00000d20       0x2e output_pic32_ssd1963\GOLMediumlFont.o
 .debug_pubnames
                0x00000d4e       0x2e output_pic32_ssd1963\GOLSmallFont.o
 .debug_pubnames
                0x00000d7c       0xe1 C:/Program Files/Microchip/mplabc32/v1.12/bin/../lib/gcc/pic32mx/3.4.4/../../../../pic32mx/lib\libc.a(ctypef.o)
 .debug_pubnames
                0x00000e5d       0x25 C:/Program Files/Microchip/mplabc32/v1.12/bin/../lib/gcc/pic32mx/3.4.4/../../../../pic32mx/lib\libc.a(puts.o)
 .debug_pubnames
                0x00000e82       0x1d C:/Program Files/Microchip/mplabc32/v1.12/bin/../lib/gcc/pic32mx/3.4.4/../../../../pic32mx/lib\libc.a(strchr.o)
 .debug_pubnames
                0x00000e9f       0x1e C:/Program Files/Microchip/mplabc32/v1.12/bin/../lib/gcc/pic32mx/3.4.4/../../../../pic32mx/lib\libc.a(strncpy.o)
 .debug_pubnames
                0x00000ebd       0x27 C:/Program Files/Microchip/mplabc32/v1.12/bin/../lib/gcc/pic32mx/3.4.4/../../../../pic32mx/lib\libc.a(printf_cdnopuxX.eo)
 .debug_pubnames
                0x00000ee4       0x21 C:/Program Files/Microchip/mplabc32/v1.12/bin/../lib/gcc/pic32mx/3.4.4/../../../../pic32mx/lib\libc.a(sprintf_s.eo)
 .debug_pubnames
                0x00000f05       0x31 C:/Program Files/Microchip/mplabc32/v1.12/bin/../lib/gcc/pic32mx/3.4.4/../../../../pic32mx/lib\libc.a(default-general-exception-handler.o)
 .debug_pubnames
                0x00000f36       0x33 C:/Program Files/Microchip/mplabc32/v1.12/bin/../lib/gcc/pic32mx/3.4.4/../../../../pic32mx/lib\libc.a(default-bootstrap-exception-handler.o)
 .debug_pubnames
                0x00000f69       0x20 C:/Program Files/Microchip/mplabc32/v1.12/bin/../lib/gcc/pic32mx/3.4.4/../../../../pic32mx/lib\libc.a(default-on-reset.o)
 .debug_pubnames
                0x00000f89       0x24 C:/Program Files/Microchip/mplabc32/v1.12/bin/../lib/gcc/pic32mx/3.4.4/../../../../pic32mx/lib\libc.a(default-on-bootstrap.o)
 .debug_pubnames
                0x00000fad       0x49 C:/Program Files/Microchip/mplabc32/v1.12/bin/../lib/gcc/pic32mx/3.4.4/../../../../pic32mx/lib\libc.a(_iob.o)
 .debug_pubnames
                0x00000ff6       0x1c C:/Program Files/Microchip/mplabc32/v1.12/bin/../lib/gcc/pic32mx/3.4.4/../../../../pic32mx/lib\libc.a(_fputc_simple.o)
 .debug_pubnames
                0x00001012       0x1d C:/Program Files/Microchip/mplabc32/v1.12/bin/../lib/gcc/pic32mx/3.4.4/../../../../pic32mx/lib\libc.a(ctype.o)
 .debug_pubnames
                0x0000102f       0x1c C:/Program Files/Microchip/mplabc32/v1.12/bin/../lib/gcc/pic32mx/3.4.4/../../../../pic32mx/lib\libc.a(write.o)
 .debug_pubnames
                0x0000104b       0x1e C:/Program Files/Microchip/mplabc32/v1.12/bin/../lib/gcc/pic32mx/3.4.4/../../../../pic32mx/lib\libc.a(_flsbuf_simple.o)
 .debug_pubnames
                0x00001069       0x20 C:/Program Files/Microchip/mplabc32/v1.12/bin/../lib/gcc/pic32mx/3.4.4/../../../../pic32mx/lib\libc.a(_mon_putc.o)
 .debug_pubnames
                0x00001089       0x21 C:/Program Files/Microchip/mplabc32/v1.12/bin/../lib/gcc/pic32mx/3.4.4/../../../../pic32mx/lib\libc.a(c32_uart.o)
 .debug_pubnames
                0x000010aa       0x24 C:/Program Files/Microchip/mplabc32/v1.12/bin/../lib/gcc/pic32mx/3.4.4/../../../../pic32mx/lib\libmchp_peripheral.a(open_core_timer_lib.o)
 .debug_pubnames
                0x000010ce       0x3b C:/Program Files/Microchip/mplabc32/v1.12/bin/../lib/gcc/pic32mx/3.4.4/../../../../pic32mx/lib\libmchp_peripheral_32MX360F512L.a(pcache.o)
 .debug_pubnames
                0x00001109       0x2b C:/Program Files/Microchip/mplabc32/v1.12/bin/../lib/gcc/pic32mx/3.4.4/../../../../pic32mx/lib\libmchp_peripheral_32MX360F512L.a(int_disable_interrupts_lib.o)
 .debug_pubnames
                0x00001134       0x2b C:/Program Files/Microchip/mplabc32/v1.12/bin/../lib/gcc/pic32mx/3.4.4/../../../../pic32mx/lib\libmchp_peripheral_32MX360F512L.a(int_restore_interrupts_lib.o)
 .debug_pubnames
                0x0000115f       0x36 C:/Program Files/Microchip/mplabc32/v1.12/bin/../lib/gcc/pic32mx/3.4.4/../../../../pic32mx/lib\libmchp_peripheral_32MX360F512L.a(int_enable_mv_int_lib.o)
 .debug_pubnames
                0x00001195       0x1f C:/Program Files/Microchip/mplabc32/v1.12/bin/../lib/gcc/pic32mx/3.4.4/../../../../pic32mx/lib\libmchp_peripheral_32MX360F512L.a(spi_getc_spi2_lib_legacy.o)
 .debug_pubnames
                0x000011b4       0x1f C:/Program Files/Microchip/mplabc32/v1.12/bin/../lib/gcc/pic32mx/3.4.4/../../../../pic32mx/lib\libmchp_peripheral_32MX360F512L.a(spi_open_spi2_lib_legacy.o)
 .debug_pubnames
                0x000011d3       0x2a C:/Program Files/Microchip/mplabc32/v1.12/bin/../lib/gcc/pic32mx/3.4.4/../../../../pic32mx/lib\libmchp_peripheral_32MX360F512L.a(int_enable_interrupts_lib.o)
 .debug_pubnames
                0x000011fd       0x2a C:/Program Files/Microchip/mplabc32/v1.12/bin/../lib/gcc/pic32mx/3.4.4/../../../../pic32mx/lib\libc.a(doprnt_cdnopsuxX.eo)

.debug_info     0x00000000     0xbf5a
 *(.debug_info .gnu.linkonce.wi.*)
 .debug_info    0x00000000      0xcc8 output_pic32_ssd1963\Application.o
 .debug_info    0x00000cc8     0x11a7 output_pic32_ssd1963\Primitive.o
 .debug_info    0x00001e6f      0x4ba output_pic32_ssd1963\GOLFontDefault.o
 .debug_info    0x00002329     0x125e output_pic32_ssd1963\JpegDecoder.o
 .debug_info    0x00003587      0xb4c output_pic32_ssd1963\BmpDecoder.o
 .debug_info    0x000040d3      0xd90 output_pic32_ssd1963\GifDecoder.o
 .debug_info    0x00004e63      0xa0b output_pic32_ssd1963\ImageDecoder.o
 .debug_info    0x0000586e      0x1f7 output_pic32_ssd1963\jidctint.o
 .debug_info    0x00005a65      0xe51 output_pic32_ssd1963\DisplayDriver.o
 .debug_info    0x000068b6      0xcbb output_pic32_ssd1963\SD-SPI.o
 .debug_info    0x00007571     0x2e2b output_pic32_ssd1963\FSIO.o
 .debug_info    0x0000a39c      0x483 output_pic32_ssd1963\GOLMediumlFont.o
 .debug_info    0x0000a81f      0x483 output_pic32_ssd1963\GOLSmallFont.o
 .debug_info    0x0000aca2      0x2e5 C:/Program Files/Microchip/mplabc32/v1.12/bin/../lib/gcc/pic32mx/3.4.4/../../../../pic32mx/lib\libc.a(ctypef.o)
 .debug_info    0x0000af87      0x158 C:/Program Files/Microchip/mplabc32/v1.12/bin/../lib/gcc/pic32mx/3.4.4/../../../../pic32mx/lib\libc.a(puts.o)
 .debug_info    0x0000b0df       0x88 C:/Program Files/Microchip/mplabc32/v1.12/bin/../lib/gcc/pic32mx/3.4.4/../../../../pic32mx/lib\libc.a(strchr.o)
 .debug_info    0x0000b167       0xab C:/Program Files/Microchip/mplabc32/v1.12/bin/../lib/gcc/pic32mx/3.4.4/../../../../pic32mx/lib\libc.a(strncpy.o)
 .debug_info    0x0000b212      0x13e C:/Program Files/Microchip/mplabc32/v1.12/bin/../lib/gcc/pic32mx/3.4.4/../../../../pic32mx/lib\libc.a(printf_cdnopuxX.eo)
 .debug_info    0x0000b350      0x13b C:/Program Files/Microchip/mplabc32/v1.12/bin/../lib/gcc/pic32mx/3.4.4/../../../../pic32mx/lib\libc.a(sprintf_s.eo)
 .debug_info    0x0000b48b       0x31 C:/Program Files/Microchip/mplabc32/v1.12/bin/../lib/gcc/pic32mx/3.4.4/../../../../pic32mx/lib\libc.a(default-general-exception-handler.o)
 .debug_info    0x0000b4bc       0x31 C:/Program Files/Microchip/mplabc32/v1.12/bin/../lib/gcc/pic32mx/3.4.4/../../../../pic32mx/lib\libc.a(default-bootstrap-exception-handler.o)
 .debug_info    0x0000b4ed       0x31 C:/Program Files/Microchip/mplabc32/v1.12/bin/../lib/gcc/pic32mx/3.4.4/../../../../pic32mx/lib\libc.a(default-on-reset.o)
 .debug_info    0x0000b51e       0x31 C:/Program Files/Microchip/mplabc32/v1.12/bin/../lib/gcc/pic32mx/3.4.4/../../../../pic32mx/lib\libc.a(default-on-bootstrap.o)
 .debug_info    0x0000b54f      0x150 C:/Program Files/Microchip/mplabc32/v1.12/bin/../lib/gcc/pic32mx/3.4.4/../../../../pic32mx/lib\libc.a(_iob.o)
 .debug_info    0x0000b69f      0x12a C:/Program Files/Microchip/mplabc32/v1.12/bin/../lib/gcc/pic32mx/3.4.4/../../../../pic32mx/lib\libc.a(_fputc_simple.o)
 .debug_info    0x0000b7c9       0x61 C:/Program Files/Microchip/mplabc32/v1.12/bin/../lib/gcc/pic32mx/3.4.4/../../../../pic32mx/lib\libc.a(ctype.o)
 .debug_info    0x0000b82a       0x7c C:/Program Files/Microchip/mplabc32/v1.12/bin/../lib/gcc/pic32mx/3.4.4/../../../../pic32mx/lib\libc.a(write.o)
 .debug_info    0x0000b8a6      0x122 C:/Program Files/Microchip/mplabc32/v1.12/bin/../lib/gcc/pic32mx/3.4.4/../../../../pic32mx/lib\libc.a(_flsbuf_simple.o)
 .debug_info    0x0000b9c8       0xfb C:/Program Files/Microchip/mplabc32/v1.12/bin/../lib/gcc/pic32mx/3.4.4/../../../../pic32mx/lib\libc.a(_mon_putc.o)
 .debug_info    0x0000bac3       0x3f C:/Program Files/Microchip/mplabc32/v1.12/bin/../lib/gcc/pic32mx/3.4.4/../../../../pic32mx/lib\libc.a(c32_uart.o)
 .debug_info    0x0000bb02       0x30 C:/Program Files/Microchip/mplabc32/v1.12/bin/../lib/gcc/pic32mx/3.4.4/../../../../pic32mx/lib\libmchp_peripheral.a(open_core_timer_lib.o)
 .debug_info    0x0000bb32       0x42 C:/Program Files/Microchip/mplabc32/v1.12/bin/../lib/gcc/pic32mx/3.4.4/../../../../pic32mx/lib\libmchp_peripheral_32MX360F512L.a(pcache.o)
 .debug_info    0x0000bb74       0x30 C:/Program Files/Microchip/mplabc32/v1.12/bin/../lib/gcc/pic32mx/3.4.4/../../../../pic32mx/lib\libmchp_peripheral_32MX360F512L.a(int_disable_interrupts_lib.o)
 .debug_info    0x0000bba4       0x30 C:/Program Files/Microchip/mplabc32/v1.12/bin/../lib/gcc/pic32mx/3.4.4/../../../../pic32mx/lib\libmchp_peripheral_32MX360F512L.a(int_restore_interrupts_lib.o)
 .debug_info    0x0000bbd4       0x30 C:/Program Files/Microchip/mplabc32/v1.12/bin/../lib/gcc/pic32mx/3.4.4/../../../../pic32mx/lib\libmchp_peripheral_32MX360F512L.a(int_enable_mv_int_lib.o)
 .debug_info    0x0000bc04       0x30 C:/Program Files/Microchip/mplabc32/v1.12/bin/../lib/gcc/pic32mx/3.4.4/../../../../pic32mx/lib\libmchp_peripheral_32MX360F512L.a(spi_getc_spi2_lib_legacy.o)
 .debug_info    0x0000bc34       0x30 C:/Program Files/Microchip/mplabc32/v1.12/bin/../lib/gcc/pic32mx/3.4.4/../../../../pic32mx/lib\libmchp_peripheral_32MX360F512L.a(spi_open_spi2_lib_legacy.o)
 .debug_info    0x0000bc64        0x0 C:/Program Files/Microchip/mplabc32/v1.12/bin/../lib/gcc/pic32mx/3.4.4/../../../../pic32mx/lib\libmchp_peripheral_32MX360F512L.a(spi_brg_tbl_lib_legacy.o)
 .debug_info    0x0000bc64       0x30 C:/Program Files/Microchip/mplabc32/v1.12/bin/../lib/gcc/pic32mx/3.4.4/../../../../pic32mx/lib\libmchp_peripheral_32MX360F512L.a(int_enable_interrupts_lib.o)
 .debug_info    0x0000bc94      0x2c6 C:/Program Files/Microchip/mplabc32/v1.12/bin/../lib/gcc/pic32mx/3.4.4/../../../../pic32mx/lib\libc.a(doprnt_cdnopsuxX.eo)

.debug_abbrev   0x00000000     0x24c4
 *(.debug_abbrev)
 .debug_abbrev  0x00000000      0x2ee output_pic32_ssd1963\Application.o
 .debug_abbrev  0x000002ee      0x296 output_pic32_ssd1963\Primitive.o
 .debug_abbrev  0x00000584      0x164 output_pic32_ssd1963\GOLFontDefault.o
 .debug_abbrev  0x000006e8      0x25a output_pic32_ssd1963\JpegDecoder.o
 .debug_abbrev  0x00000942      0x229 output_pic32_ssd1963\BmpDecoder.o
 .debug_abbrev  0x00000b6b      0x26a output_pic32_ssd1963\GifDecoder.o
 .debug_abbrev  0x00000dd5      0x23f output_pic32_ssd1963\ImageDecoder.o
 .debug_abbrev  0x00001014       0x9d output_pic32_ssd1963\jidctint.o
 .debug_abbrev  0x000010b1      0x25e output_pic32_ssd1963\DisplayDriver.o
 .debug_abbrev  0x0000130f      0x2d4 output_pic32_ssd1963\SD-SPI.o
 .debug_abbrev  0x000015e3      0x2a1 output_pic32_ssd1963\FSIO.o
 .debug_abbrev  0x00001884      0x145 output_pic32_ssd1963\GOLMediumlFont.o
 .debug_abbrev  0x000019c9      0x145 output_pic32_ssd1963\GOLSmallFont.o
 .debug_abbrev  0x00001b0e       0x74 C:/Program Files/Microchip/mplabc32/v1.12/bin/../lib/gcc/pic32mx/3.4.4/../../../../pic32mx/lib\libc.a(ctypef.o)
 .debug_abbrev  0x00001b82       0xb9 C:/Program Files/Microchip/mplabc32/v1.12/bin/../lib/gcc/pic32mx/3.4.4/../../../../pic32mx/lib\libc.a(puts.o)
 .debug_abbrev  0x00001c3b       0x5e C:/Program Files/Microchip/mplabc32/v1.12/bin/../lib/gcc/pic32mx/3.4.4/../../../../pic32mx/lib\libc.a(strchr.o)
 .debug_abbrev  0x00001c99       0x89 C:/Program Files/Microchip/mplabc32/v1.12/bin/../lib/gcc/pic32mx/3.4.4/../../../../pic32mx/lib\libc.a(strncpy.o)
 .debug_abbrev  0x00001d22       0xc7 C:/Program Files/Microchip/mplabc32/v1.12/bin/../lib/gcc/pic32mx/3.4.4/../../../../pic32mx/lib\libc.a(printf_cdnopuxX.eo)
 .debug_abbrev  0x00001de9       0xb3 C:/Program Files/Microchip/mplabc32/v1.12/bin/../lib/gcc/pic32mx/3.4.4/../../../../pic32mx/lib\libc.a(sprintf_s.eo)
 .debug_abbrev  0x00001e9c       0x25 C:/Program Files/Microchip/mplabc32/v1.12/bin/../lib/gcc/pic32mx/3.4.4/../../../../pic32mx/lib\libc.a(default-general-exception-handler.o)
 .debug_abbrev  0x00001ec1       0x25 C:/Program Files/Microchip/mplabc32/v1.12/bin/../lib/gcc/pic32mx/3.4.4/../../../../pic32mx/lib\libc.a(default-bootstrap-exception-handler.o)
 .debug_abbrev  0x00001ee6       0x25 C:/Program Files/Microchip/mplabc32/v1.12/bin/../lib/gcc/pic32mx/3.4.4/../../../../pic32mx/lib\libc.a(default-on-reset.o)
 .debug_abbrev  0x00001f0b       0x25 C:/Program Files/Microchip/mplabc32/v1.12/bin/../lib/gcc/pic32mx/3.4.4/../../../../pic32mx/lib\libc.a(default-on-bootstrap.o)
 .debug_abbrev  0x00001f30       0x81 C:/Program Files/Microchip/mplabc32/v1.12/bin/../lib/gcc/pic32mx/3.4.4/../../../../pic32mx/lib\libc.a(_iob.o)
 .debug_abbrev  0x00001fb1       0xb4 C:/Program Files/Microchip/mplabc32/v1.12/bin/../lib/gcc/pic32mx/3.4.4/../../../../pic32mx/lib\libc.a(_fputc_simple.o)
 .debug_abbrev  0x00002065       0x49 C:/Program Files/Microchip/mplabc32/v1.12/bin/../lib/gcc/pic32mx/3.4.4/../../../../pic32mx/lib\libc.a(ctype.o)
 .debug_abbrev  0x000020ae       0x73 C:/Program Files/Microchip/mplabc32/v1.12/bin/../lib/gcc/pic32mx/3.4.4/../../../../pic32mx/lib\libc.a(write.o)
 .debug_abbrev  0x00002121       0xa7 C:/Program Files/Microchip/mplabc32/v1.12/bin/../lib/gcc/pic32mx/3.4.4/../../../../pic32mx/lib\libc.a(_flsbuf_simple.o)
 .debug_abbrev  0x000021c8       0x89 C:/Program Files/Microchip/mplabc32/v1.12/bin/../lib/gcc/pic32mx/3.4.4/../../../../pic32mx/lib\libc.a(_mon_putc.o)
 .debug_abbrev  0x00002251       0x30 C:/Program Files/Microchip/mplabc32/v1.12/bin/../lib/gcc/pic32mx/3.4.4/../../../../pic32mx/lib\libc.a(c32_uart.o)
 .debug_abbrev  0x00002281       0x23 C:/Program Files/Microchip/mplabc32/v1.12/bin/../lib/gcc/pic32mx/3.4.4/../../../../pic32mx/lib\libmchp_peripheral.a(open_core_timer_lib.o)
 .debug_abbrev  0x000022a4       0x23 C:/Program Files/Microchip/mplabc32/v1.12/bin/../lib/gcc/pic32mx/3.4.4/../../../../pic32mx/lib\libmchp_peripheral_32MX360F512L.a(pcache.o)
 .debug_abbrev  0x000022c7       0x23 C:/Program Files/Microchip/mplabc32/v1.12/bin/../lib/gcc/pic32mx/3.4.4/../../../../pic32mx/lib\libmchp_peripheral_32MX360F512L.a(int_disable_interrupts_lib.o)
 .debug_abbrev  0x000022ea       0x23 C:/Program Files/Microchip/mplabc32/v1.12/bin/../lib/gcc/pic32mx/3.4.4/../../../../pic32mx/lib\libmchp_peripheral_32MX360F512L.a(int_restore_interrupts_lib.o)
 .debug_abbrev  0x0000230d       0x23 C:/Program Files/Microchip/mplabc32/v1.12/bin/../lib/gcc/pic32mx/3.4.4/../../../../pic32mx/lib\libmchp_peripheral_32MX360F512L.a(int_enable_mv_int_lib.o)
 .debug_abbrev  0x00002330       0x23 C:/Program Files/Microchip/mplabc32/v1.12/bin/../lib/gcc/pic32mx/3.4.4/../../../../pic32mx/lib\libmchp_peripheral_32MX360F512L.a(spi_getc_spi2_lib_legacy.o)
 .debug_abbrev  0x00002353       0x23 C:/Program Files/Microchip/mplabc32/v1.12/bin/../lib/gcc/pic32mx/3.4.4/../../../../pic32mx/lib\libmchp_peripheral_32MX360F512L.a(spi_open_spi2_lib_legacy.o)
 .debug_abbrev  0x00002376        0x1 C:/Program Files/Microchip/mplabc32/v1.12/bin/../lib/gcc/pic32mx/3.4.4/../../../../pic32mx/lib\libmchp_peripheral_32MX360F512L.a(spi_brg_tbl_lib_legacy.o)
 .debug_abbrev  0x00002377       0x23 C:/Program Files/Microchip/mplabc32/v1.12/bin/../lib/gcc/pic32mx/3.4.4/../../../../pic32mx/lib\libmchp_peripheral_32MX360F512L.a(int_enable_interrupts_lib.o)
 .debug_abbrev  0x0000239a      0x12a C:/Program Files/Microchip/mplabc32/v1.12/bin/../lib/gcc/pic32mx/3.4.4/../../../../pic32mx/lib\libc.a(doprnt_cdnopsuxX.eo)

.debug_line     0x00000000     0x5b71
 *(.debug_line)
 .debug_line    0x00000000      0x440 output_pic32_ssd1963\Application.o
 .debug_line    0x00000440      0x507 output_pic32_ssd1963\Primitive.o
 .debug_line    0x00000947      0x192 output_pic32_ssd1963\GOLFontDefault.o
 .debug_line    0x00000ad9      0x5d8 output_pic32_ssd1963\JpegDecoder.o
 .debug_line    0x000010b1      0x4e6 output_pic32_ssd1963\BmpDecoder.o
 .debug_line    0x00001597      0x475 output_pic32_ssd1963\GifDecoder.o
 .debug_line    0x00001a0c      0x2c8 output_pic32_ssd1963\ImageDecoder.o
 .debug_line    0x00001cd4      0x172 output_pic32_ssd1963\jidctint.o
 .debug_line    0x00001e46      0x4bb output_pic32_ssd1963\DisplayDriver.o
 .debug_line    0x00002301      0x360 output_pic32_ssd1963\SD-SPI.o
 .debug_line    0x00002661     0x13fe output_pic32_ssd1963\FSIO.o
 .debug_line    0x00003a5f      0x164 output_pic32_ssd1963\GOLMediumlFont.o
 .debug_line    0x00003bc3      0x162 output_pic32_ssd1963\GOLSmallFont.o
 .debug_line    0x00003d25      0x254 C:/Program Files/Microchip/mplabc32/v1.12/bin/../lib/gcc/pic32mx/3.4.4/../../../../pic32mx/lib\libc.a(ctypef.o)
 .debug_line    0x00003f79      0x1cf C:/Program Files/Microchip/mplabc32/v1.12/bin/../lib/gcc/pic32mx/3.4.4/../../../../pic32mx/lib\libc.a(puts.o)
 .debug_line    0x00004148      0x1a0 C:/Program Files/Microchip/mplabc32/v1.12/bin/../lib/gcc/pic32mx/3.4.4/../../../../pic32mx/lib\libc.a(strchr.o)
 .debug_line    0x000042e8      0x1a7 C:/Program Files/Microchip/mplabc32/v1.12/bin/../lib/gcc/pic32mx/3.4.4/../../../../pic32mx/lib\libc.a(strncpy.o)
 .debug_line    0x0000448f      0x161 C:/Program Files/Microchip/mplabc32/v1.12/bin/../lib/gcc/pic32mx/3.4.4/../../../../pic32mx/lib\libc.a(printf_cdnopuxX.eo)
 .debug_line    0x000045f0      0x172 C:/Program Files/Microchip/mplabc32/v1.12/bin/../lib/gcc/pic32mx/3.4.4/../../../../pic32mx/lib\libc.a(sprintf_s.eo)
 .debug_line    0x00004762       0xba C:/Program Files/Microchip/mplabc32/v1.12/bin/../lib/gcc/pic32mx/3.4.4/../../../../pic32mx/lib\libc.a(default-general-exception-handler.o)
 .debug_line    0x0000481c       0xbc C:/Program Files/Microchip/mplabc32/v1.12/bin/../lib/gcc/pic32mx/3.4.4/../../../../pic32mx/lib\libc.a(default-bootstrap-exception-handler.o)
 .debug_line    0x000048d8       0xa9 C:/Program Files/Microchip/mplabc32/v1.12/bin/../lib/gcc/pic32mx/3.4.4/../../../../pic32mx/lib\libc.a(default-on-reset.o)
 .debug_line    0x00004981       0xad C:/Program Files/Microchip/mplabc32/v1.12/bin/../lib/gcc/pic32mx/3.4.4/../../../../pic32mx/lib\libc.a(default-on-bootstrap.o)
 .debug_line    0x00004a2e      0x196 C:/Program Files/Microchip/mplabc32/v1.12/bin/../lib/gcc/pic32mx/3.4.4/../../../../pic32mx/lib\libc.a(_iob.o)
 .debug_line    0x00004bc4      0x197 C:/Program Files/Microchip/mplabc32/v1.12/bin/../lib/gcc/pic32mx/3.4.4/../../../../pic32mx/lib\libc.a(_fputc_simple.o)
 .debug_line    0x00004d5b      0x102 C:/Program Files/Microchip/mplabc32/v1.12/bin/../lib/gcc/pic32mx/3.4.4/../../../../pic32mx/lib\libc.a(ctype.o)
 .debug_line    0x00004e5d       0xc2 C:/Program Files/Microchip/mplabc32/v1.12/bin/../lib/gcc/pic32mx/3.4.4/../../../../pic32mx/lib\libc.a(write.o)
 .debug_line    0x00004f1f      0x19d C:/Program Files/Microchip/mplabc32/v1.12/bin/../lib/gcc/pic32mx/3.4.4/../../../../pic32mx/lib\libc.a(_flsbuf_simple.o)
 .debug_line    0x000050bc       0xd3 C:/Program Files/Microchip/mplabc32/v1.12/bin/../lib/gcc/pic32mx/3.4.4/../../../../pic32mx/lib\libc.a(_mon_putc.o)
 .debug_line    0x0000518f       0x8f C:/Program Files/Microchip/mplabc32/v1.12/bin/../lib/gcc/pic32mx/3.4.4/../../../../pic32mx/lib\libc.a(c32_uart.o)
 .debug_line    0x0000521e       0xa9 C:/Program Files/Microchip/mplabc32/v1.12/bin/../lib/gcc/pic32mx/3.4.4/../../../../pic32mx/lib\libmchp_peripheral.a(open_core_timer_lib.o)
 .debug_line    0x000052c7       0x9d C:/Program Files/Microchip/mplabc32/v1.12/bin/../lib/gcc/pic32mx/3.4.4/../../../../pic32mx/lib\libmchp_peripheral_32MX360F512L.a(pcache.o)
 .debug_line    0x00005364       0xae C:/Program Files/Microchip/mplabc32/v1.12/bin/../lib/gcc/pic32mx/3.4.4/../../../../pic32mx/lib\libmchp_peripheral_32MX360F512L.a(int_disable_interrupts_lib.o)
 .debug_line    0x00005412       0xae C:/Program Files/Microchip/mplabc32/v1.12/bin/../lib/gcc/pic32mx/3.4.4/../../../../pic32mx/lib\libmchp_peripheral_32MX360F512L.a(int_restore_interrupts_lib.o)
 .debug_line    0x000054c0       0xa9 C:/Program Files/Microchip/mplabc32/v1.12/bin/../lib/gcc/pic32mx/3.4.4/../../../../pic32mx/lib\libmchp_peripheral_32MX360F512L.a(int_enable_mv_int_lib.o)
 .debug_line    0x00005569       0xac C:/Program Files/Microchip/mplabc32/v1.12/bin/../lib/gcc/pic32mx/3.4.4/../../../../pic32mx/lib\libmchp_peripheral_32MX360F512L.a(spi_getc_spi2_lib_legacy.o)
 .debug_line    0x00005615       0xac C:/Program Files/Microchip/mplabc32/v1.12/bin/../lib/gcc/pic32mx/3.4.4/../../../../pic32mx/lib\libmchp_peripheral_32MX360F512L.a(spi_open_spi2_lib_legacy.o)
 .debug_line    0x000056c1        0x0 C:/Program Files/Microchip/mplabc32/v1.12/bin/../lib/gcc/pic32mx/3.4.4/../../../../pic32mx/lib\libmchp_peripheral_32MX360F512L.a(spi_brg_tbl_lib_legacy.o)
 .debug_line    0x000056c1       0xad C:/Program Files/Microchip/mplabc32/v1.12/bin/../lib/gcc/pic32mx/3.4.4/../../../../pic32mx/lib\libmchp_peripheral_32MX360F512L.a(int_enable_interrupts_lib.o)
 .debug_line    0x0000576e      0x403 C:/Program Files/Microchip/mplabc32/v1.12/bin/../lib/gcc/pic32mx/3.4.4/../../../../pic32mx/lib\libc.a(doprnt_cdnopsuxX.eo)

.debug_frame    0x00000000     0x17a4
 *(.debug_frame)
 .debug_frame   0x00000000       0x5c output_pic32_ssd1963\Application.o
 .debug_frame   0x0000005c      0x1dc output_pic32_ssd1963\Primitive.o
 .debug_frame   0x00000238      0x1d4 output_pic32_ssd1963\JpegDecoder.o
 .debug_frame   0x0000040c       0x74 output_pic32_ssd1963\BmpDecoder.o
 .debug_frame   0x00000480      0x1a8 output_pic32_ssd1963\GifDecoder.o
 .debug_frame   0x00000628       0x58 output_pic32_ssd1963\ImageDecoder.o
 .debug_frame   0x00000680       0x34 output_pic32_ssd1963\jidctint.o
 .debug_frame   0x000006b4      0x2b0 output_pic32_ssd1963\DisplayDriver.o
 .debug_frame   0x00000964      0x16c output_pic32_ssd1963\SD-SPI.o
 .debug_frame   0x00000ad0      0x844 output_pic32_ssd1963\FSIO.o
 .debug_frame   0x00001314      0x120 C:/Program Files/Microchip/mplabc32/v1.12/bin/../lib/gcc/pic32mx/3.4.4/../../../../pic32mx/lib\libc.a(ctypef.o)
 .debug_frame   0x00001434       0x50 C:/Program Files/Microchip/mplabc32/v1.12/bin/../lib/gcc/pic32mx/3.4.4/../../../../pic32mx/lib\libc.a(puts.o)
 .debug_frame   0x00001484       0x20 C:/Program Files/Microchip/mplabc32/v1.12/bin/../lib/gcc/pic32mx/3.4.4/../../../../pic32mx/lib\libc.a(strchr.o)
 .debug_frame   0x000014a4       0x20 C:/Program Files/Microchip/mplabc32/v1.12/bin/../lib/gcc/pic32mx/3.4.4/../../../../pic32mx/lib\libc.a(strncpy.o)
 .debug_frame   0x000014c4       0x28 C:/Program Files/Microchip/mplabc32/v1.12/bin/../lib/gcc/pic32mx/3.4.4/../../../../pic32mx/lib\libc.a(printf_cdnopuxX.eo)
 .debug_frame   0x000014ec       0x2c C:/Program Files/Microchip/mplabc32/v1.12/bin/../lib/gcc/pic32mx/3.4.4/../../../../pic32mx/lib\libc.a(sprintf_s.eo)
 .debug_frame   0x00001518       0x20 C:/Program Files/Microchip/mplabc32/v1.12/bin/../lib/gcc/pic32mx/3.4.4/../../../../pic32mx/lib\libc.a(default-general-exception-handler.o)
 .debug_frame   0x00001538       0x20 C:/Program Files/Microchip/mplabc32/v1.12/bin/../lib/gcc/pic32mx/3.4.4/../../../../pic32mx/lib\libc.a(default-bootstrap-exception-handler.o)
 .debug_frame   0x00001558       0x20 C:/Program Files/Microchip/mplabc32/v1.12/bin/../lib/gcc/pic32mx/3.4.4/../../../../pic32mx/lib\libc.a(default-on-reset.o)
 .debug_frame   0x00001578       0x20 C:/Program Files/Microchip/mplabc32/v1.12/bin/../lib/gcc/pic32mx/3.4.4/../../../../pic32mx/lib\libc.a(default-on-bootstrap.o)
 .debug_frame   0x00001598       0x30 C:/Program Files/Microchip/mplabc32/v1.12/bin/../lib/gcc/pic32mx/3.4.4/../../../../pic32mx/lib\libc.a(_fputc_simple.o)
 .debug_frame   0x000015c8       0x34 C:/Program Files/Microchip/mplabc32/v1.12/bin/../lib/gcc/pic32mx/3.4.4/../../../../pic32mx/lib\libc.a(write.o)
 .debug_frame   0x000015fc       0x2c C:/Program Files/Microchip/mplabc32/v1.12/bin/../lib/gcc/pic32mx/3.4.4/../../../../pic32mx/lib\libc.a(_flsbuf_simple.o)
 .debug_frame   0x00001628       0x20 C:/Program Files/Microchip/mplabc32/v1.12/bin/../lib/gcc/pic32mx/3.4.4/../../../../pic32mx/lib\libc.a(_mon_putc.o)
 .debug_frame   0x00001648       0x20 C:/Program Files/Microchip/mplabc32/v1.12/bin/../lib/gcc/pic32mx/3.4.4/../../../../pic32mx/lib\libmchp_peripheral.a(open_core_timer_lib.o)
 .debug_frame   0x00001668       0x30 C:/Program Files/Microchip/mplabc32/v1.12/bin/../lib/gcc/pic32mx/3.4.4/../../../../pic32mx/lib\libmchp_peripheral_32MX360F512L.a(pcache.o)
 .debug_frame   0x00001698       0x20 C:/Program Files/Microchip/mplabc32/v1.12/bin/../lib/gcc/pic32mx/3.4.4/../../../../pic32mx/lib\libmchp_peripheral_32MX360F512L.a(int_disable_interrupts_lib.o)
 .debug_frame   0x000016b8       0x20 C:/Program Files/Microchip/mplabc32/v1.12/bin/../lib/gcc/pic32mx/3.4.4/../../../../pic32mx/lib\libmchp_peripheral_32MX360F512L.a(int_restore_interrupts_lib.o)
 .debug_frame   0x000016d8       0x28 C:/Program Files/Microchip/mplabc32/v1.12/bin/../lib/gcc/pic32mx/3.4.4/../../../../pic32mx/lib\libmchp_peripheral_32MX360F512L.a(int_enable_mv_int_lib.o)
 .debug_frame   0x00001700       0x20 C:/Program Files/Microchip/mplabc32/v1.12/bin/../lib/gcc/pic32mx/3.4.4/../../../../pic32mx/lib\libmchp_peripheral_32MX360F512L.a(spi_getc_spi2_lib_legacy.o)
 .debug_frame   0x00001720       0x20 C:/Program Files/Microchip/mplabc32/v1.12/bin/../lib/gcc/pic32mx/3.4.4/../../../../pic32mx/lib\libmchp_peripheral_32MX360F512L.a(spi_open_spi2_lib_legacy.o)
 .debug_frame   0x00001740       0x20 C:/Program Files/Microchip/mplabc32/v1.12/bin/../lib/gcc/pic32mx/3.4.4/../../../../pic32mx/lib\libmchp_peripheral_32MX360F512L.a(int_enable_interrupts_lib.o)
 .debug_frame   0x00001760       0x44 C:/Program Files/Microchip/mplabc32/v1.12/bin/../lib/gcc/pic32mx/3.4.4/../../../../pic32mx/lib\libc.a(doprnt_cdnopsuxX.eo)

.debug_str      0x00000000     0x3927
 *(.debug_str)
 .debug_str     0x00000000      0x5be output_pic32_ssd1963\Application.o
                                0x6a3 (size before relaxing)
 .debug_str     0x000005be      0x2b3 output_pic32_ssd1963\Primitive.o
                                0x612 (size before relaxing)
 .debug_str     0x00000871       0x2e output_pic32_ssd1963\GOLFontDefault.o
                                0x35c (size before relaxing)
 .debug_str     0x0000089f      0x5a5 output_pic32_ssd1963\JpegDecoder.o
                                0x9b9 (size before relaxing)
 .debug_str     0x00000e44      0x17d output_pic32_ssd1963\BmpDecoder.o
                                0x601 (size before relaxing)
 .debug_str     0x00000fc1      0x3ac output_pic32_ssd1963\GifDecoder.o
                                0x867 (size before relaxing)
 .debug_str     0x0000136d      0x142 output_pic32_ssd1963\ImageDecoder.o
                                0x67e (size before relaxing)
 .debug_str     0x000014af       0x95 output_pic32_ssd1963\jidctint.o
                                0x197 (size before relaxing)
 .debug_str     0x00001544      0x2e2 output_pic32_ssd1963\DisplayDriver.o
                                0x66d (size before relaxing)
 .debug_str     0x00001826      0x419 output_pic32_ssd1963\SD-SPI.o
                                0x7a0 (size before relaxing)
 .debug_str     0x00001c3f      0xec6 output_pic32_ssd1963\FSIO.o
                               0x13e8 (size before relaxing)
 .debug_str     0x00002b05       0x3b output_pic32_ssd1963\GOLMediumlFont.o
                                0x31e (size before relaxing)
 .debug_str     0x00002b40       0x2c output_pic32_ssd1963\GOLSmallFont.o
                                0x31c (size before relaxing)
 .debug_str     0x00002b6c       0xef C:/Program Files/Microchip/mplabc32/v1.12/bin/../lib/gcc/pic32mx/3.4.4/../../../../pic32mx/lib\libc.a(ctypef.o)
                                0x14b (size before relaxing)
 .debug_str     0x00002c5b       0x99 C:/Program Files/Microchip/mplabc32/v1.12/bin/../lib/gcc/pic32mx/3.4.4/../../../../pic32mx/lib\libc.a(puts.o)
                                0x13c (size before relaxing)
 .debug_str     0x00002cf4       0x74 C:/Program Files/Microchip/mplabc32/v1.12/bin/../lib/gcc/pic32mx/3.4.4/../../../../pic32mx/lib\libc.a(strchr.o)
                                 0xe8 (size before relaxing)
 .debug_str     0x00002d68       0x7b C:/Program Files/Microchip/mplabc32/v1.12/bin/../lib/gcc/pic32mx/3.4.4/../../../../pic32mx/lib\libc.a(strncpy.o)
                                 0xfb (size before relaxing)
 .debug_str     0x00002de3       0x8f C:/Program Files/Microchip/mplabc32/v1.12/bin/../lib/gcc/pic32mx/3.4.4/../../../../pic32mx/lib\libc.a(printf_cdnopuxX.eo)
                                0x15d (size before relaxing)
 .debug_str     0x00002e72       0x1c C:/Program Files/Microchip/mplabc32/v1.12/bin/../lib/gcc/pic32mx/3.4.4/../../../../pic32mx/lib\libc.a(sprintf_s.eo)
                                0x153 (size before relaxing)
 .debug_str     0x00002e8e       0xa5 C:/Program Files/Microchip/mplabc32/v1.12/bin/../lib/gcc/pic32mx/3.4.4/../../../../pic32mx/lib\libc.a(default-general-exception-handler.o)
                                 0xec (size before relaxing)
 .debug_str     0x00002f33       0xa9 C:/Program Files/Microchip/mplabc32/v1.12/bin/../lib/gcc/pic32mx/3.4.4/../../../../pic32mx/lib\libc.a(default-bootstrap-exception-handler.o)
                                 0xf0 (size before relaxing)
 .debug_str     0x00002fdc       0x83 C:/Program Files/Microchip/mplabc32/v1.12/bin/../lib/gcc/pic32mx/3.4.4/../../../../pic32mx/lib\libc.a(default-on-reset.o)
                                 0xca (size before relaxing)
 .debug_str     0x0000305f       0x8b C:/Program Files/Microchip/mplabc32/v1.12/bin/../lib/gcc/pic32mx/3.4.4/../../../../pic32mx/lib\libc.a(default-on-bootstrap.o)
                                 0xd2 (size before relaxing)
 .debug_str     0x000030ea       0x89 C:/Program Files/Microchip/mplabc32/v1.12/bin/../lib/gcc/pic32mx/3.4.4/../../../../pic32mx/lib\libc.a(_iob.o)
                                0x14f (size before relaxing)
 .debug_str     0x00003173       0x15 C:/Program Files/Microchip/mplabc32/v1.12/bin/../lib/gcc/pic32mx/3.4.4/../../../../pic32mx/lib\libc.a(_fputc_simple.o)
                                0x149 (size before relaxing)
 .debug_str     0x00003188       0x6c C:/Program Files/Microchip/mplabc32/v1.12/bin/../lib/gcc/pic32mx/3.4.4/../../../../pic32mx/lib\libc.a(ctype.o)
                                 0xd1 (size before relaxing)
 .debug_str     0x000031f4       0x6e C:/Program Files/Microchip/mplabc32/v1.12/bin/../lib/gcc/pic32mx/3.4.4/../../../../pic32mx/lib\libc.a(write.o)
                                 0xd6 (size before relaxing)
 .debug_str     0x00003262       0x18 C:/Program Files/Microchip/mplabc32/v1.12/bin/../lib/gcc/pic32mx/3.4.4/../../../../pic32mx/lib\libc.a(_flsbuf_simple.o)
                                0x144 (size before relaxing)
 .debug_str     0x0000327a       0xdb C:/Program Files/Microchip/mplabc32/v1.12/bin/../lib/gcc/pic32mx/3.4.4/../../../../pic32mx/lib\libc.a(_mon_putc.o)
                                0x13a (size before relaxing)
 .debug_str     0x00003355       0x6f C:/Program Files/Microchip/mplabc32/v1.12/bin/../lib/gcc/pic32mx/3.4.4/../../../../pic32mx/lib\libc.a(c32_uart.o)
                                 0xc1 (size before relaxing)
 .debug_str     0x000033c4       0x97 C:/Program Files/Microchip/mplabc32/v1.12/bin/../lib/gcc/pic32mx/3.4.4/../../../../pic32mx/lib\libmchp_peripheral.a(open_core_timer_lib.o)
                                 0xde (size before relaxing)
 .debug_str     0x0000345b       0x9e C:/Program Files/Microchip/mplabc32/v1.12/bin/../lib/gcc/pic32mx/3.4.4/../../../../pic32mx/lib\libmchp_peripheral_32MX360F512L.a(pcache.o)
                                 0xe5 (size before relaxing)
 .debug_str     0x000034f9       0xa3 C:/Program Files/Microchip/mplabc32/v1.12/bin/../lib/gcc/pic32mx/3.4.4/../../../../pic32mx/lib\libmchp_peripheral_32MX360F512L.a(int_disable_interrupts_lib.o)
                                 0xea (size before relaxing)
 .debug_str     0x0000359c       0xa3 C:/Program Files/Microchip/mplabc32/v1.12/bin/../lib/gcc/pic32mx/3.4.4/../../../../pic32mx/lib\libmchp_peripheral_32MX360F512L.a(int_restore_interrupts_lib.o)
                                 0xea (size before relaxing)
 .debug_str     0x0000363f       0xa9 C:/Program Files/Microchip/mplabc32/v1.12/bin/../lib/gcc/pic32mx/3.4.4/../../../../pic32mx/lib\libmchp_peripheral_32MX360F512L.a(int_enable_mv_int_lib.o)
                                 0xf0 (size before relaxing)
 .debug_str     0x000036e8       0x95 C:/Program Files/Microchip/mplabc32/v1.12/bin/../lib/gcc/pic32mx/3.4.4/../../../../pic32mx/lib\libmchp_peripheral_32MX360F512L.a(spi_getc_spi2_lib_legacy.o)
                                 0xdc (size before relaxing)
 .debug_str     0x0000377d       0x95 C:/Program Files/Microchip/mplabc32/v1.12/bin/../lib/gcc/pic32mx/3.4.4/../../../../pic32mx/lib\libmchp_peripheral_32MX360F512L.a(spi_open_spi2_lib_legacy.o)
                                 0xdc (size before relaxing)
 .debug_str     0x00003812       0xa1 C:/Program Files/Microchip/mplabc32/v1.12/bin/../lib/gcc/pic32mx/3.4.4/../../../../pic32mx/lib\libmchp_peripheral_32MX360F512L.a(int_enable_interrupts_lib.o)
                                 0xe8 (size before relaxing)
 .debug_str     0x000038b3       0x74 C:/Program Files/Microchip/mplabc32/v1.12/bin/../lib/gcc/pic32mx/3.4.4/../../../../pic32mx/lib\libc.a(doprnt_cdnopsuxX.eo)
                                0x1e0 (size before relaxing)

.debug_loc
 *(.debug_loc)

.debug_macinfo  0x00000000    0x15937
 *(.debug_macinfo)
 .debug_macinfo
                0x00000000      0xc8e C:/Program Files/Microchip/mplabc32/v1.12/bin/../lib/gcc/pic32mx/3.4.4/../../../../pic32mx/lib\libc.a(ctypef.o)
 .debug_macinfo
                0x00000c8e     0x1e47 C:/Program Files/Microchip/mplabc32/v1.12/bin/../lib/gcc/pic32mx/3.4.4/../../../../pic32mx/lib\libc.a(puts.o)
 .debug_macinfo
                0x00002ad5      0xae6 C:/Program Files/Microchip/mplabc32/v1.12/bin/../lib/gcc/pic32mx/3.4.4/../../../../pic32mx/lib\libc.a(strchr.o)
 .debug_macinfo
                0x000035bb      0xae6 C:/Program Files/Microchip/mplabc32/v1.12/bin/../lib/gcc/pic32mx/3.4.4/../../../../pic32mx/lib\libc.a(strncpy.o)
 .debug_macinfo
                0x000040a1     0x1fe9 C:/Program Files/Microchip/mplabc32/v1.12/bin/../lib/gcc/pic32mx/3.4.4/../../../../pic32mx/lib\libc.a(printf_cdnopuxX.eo)
 .debug_macinfo
                0x0000608a     0x2039 C:/Program Files/Microchip/mplabc32/v1.12/bin/../lib/gcc/pic32mx/3.4.4/../../../../pic32mx/lib\libc.a(sprintf_s.eo)
 .debug_macinfo
                0x000080c3      0x92f C:/Program Files/Microchip/mplabc32/v1.12/bin/../lib/gcc/pic32mx/3.4.4/../../../../pic32mx/lib\libc.a(default-general-exception-handler.o)
 .debug_macinfo
                0x000089f2      0x92f C:/Program Files/Microchip/mplabc32/v1.12/bin/../lib/gcc/pic32mx/3.4.4/../../../../pic32mx/lib\libc.a(default-bootstrap-exception-handler.o)
 .debug_macinfo
                0x00009321      0x92f C:/Program Files/Microchip/mplabc32/v1.12/bin/../lib/gcc/pic32mx/3.4.4/../../../../pic32mx/lib\libc.a(default-on-reset.o)
 .debug_macinfo
                0x00009c50      0x92f C:/Program Files/Microchip/mplabc32/v1.12/bin/../lib/gcc/pic32mx/3.4.4/../../../../pic32mx/lib\libc.a(default-on-bootstrap.o)
 .debug_macinfo
                0x0000a57f     0x1e4e C:/Program Files/Microchip/mplabc32/v1.12/bin/../lib/gcc/pic32mx/3.4.4/../../../../pic32mx/lib\libc.a(_iob.o)
 .debug_macinfo
                0x0000c3cd     0x1e8f C:/Program Files/Microchip/mplabc32/v1.12/bin/../lib/gcc/pic32mx/3.4.4/../../../../pic32mx/lib\libc.a(_fputc_simple.o)
 .debug_macinfo
                0x0000e25c      0xcd9 C:/Program Files/Microchip/mplabc32/v1.12/bin/../lib/gcc/pic32mx/3.4.4/../../../../pic32mx/lib\libc.a(ctype.o)
 .debug_macinfo
                0x0000ef35      0x92f C:/Program Files/Microchip/mplabc32/v1.12/bin/../lib/gcc/pic32mx/3.4.4/../../../../pic32mx/lib\libc.a(write.o)
 .debug_macinfo
                0x0000f864     0x1eb3 C:/Program Files/Microchip/mplabc32/v1.12/bin/../lib/gcc/pic32mx/3.4.4/../../../../pic32mx/lib\libc.a(_flsbuf_simple.o)
 .debug_macinfo
                0x00011717      0x9bc C:/Program Files/Microchip/mplabc32/v1.12/bin/../lib/gcc/pic32mx/3.4.4/../../../../pic32mx/lib\libc.a(_mon_putc.o)
 .debug_macinfo
                0x000120d3      0x92f C:/Program Files/Microchip/mplabc32/v1.12/bin/../lib/gcc/pic32mx/3.4.4/../../../../pic32mx/lib\libc.a(c32_uart.o)
 .debug_macinfo
                0x00012a02     0x2f35 C:/Program Files/Microchip/mplabc32/v1.12/bin/../lib/gcc/pic32mx/3.4.4/../../../../pic32mx/lib\libc.a(doprnt_cdnopsuxX.eo)

.debug_weaknames
 *(.debug_weaknames)

.debug_funcnames
 *(.debug_funcnames)

.debug_typenames
 *(.debug_typenames)

.debug_varnames
 *(.debug_varnames)
OUTPUT(output_pic32_ssd1963\ImageFromSD SSD1963 PIC32.elf elf32-tradlittlemips)

.debug_ranges   0x00000000       0x78
 .debug_ranges  0x00000000       0x48 output_pic32_ssd1963\BmpDecoder.o
 .debug_ranges  0x00000048       0x18 output_pic32_ssd1963\GifDecoder.o
 .debug_ranges  0x00000060       0x18 output_pic32_ssd1963\FSIO.o
